:020000040800F2
:1000000000000220317D0008A17B0008A37B0008CE
:10001000A57B0008A77B0008A97B00080000000062
:10002000000000000000000000000000AB7B0008A2
:10003000AD7B000800000000AF7B0008B17B00082A
:10004000817D0008817D0008817D0008817D000898
:10005000817D0008817D0008817D0008817D000888
:10006000817D0008817D0008817D0008817D000878
:10007000817D0008817D0008817D0008817D000868
:10008000817D0008817D0008817D0008817D000858
:10009000817D0008817D0008817D0008817D000848
:1000A000817D0008817D0008817D0008817D000838
:1000B000817D0008817D0008817D0008817D000828
:1000C000817D0008817D0008817D0008817D000818
:1000D000817D0008B57B0008817D0008C17B000898
:1000E000817D0008817D0008817D0008817D0008F8
:1000F000817D0008817D0008817D0008817D0008E8
:10010000817D0008817D0008817D0008817D0008D7
:10011000817D0008817D0008F17B0008817D000859
:10012000817D0008817D0008817D0008817D0008B7
:10013000817D0008817D0008817D0008817D0008A7
:10014000817D0008817D0008817D0008817D000897
:10015000817D0008817D0008817D0008817D000887
:10016000817D0008817D0008817D0008817D000877
:10017000817D0008817D0008817D0008000000006D
:04018000817D000875
:1001840010B5054C237833B9044B13B10448AFF3CD
:1001940000800123237010BD6800002000000000CF
:1001A400D891000808B5034B1BB103490348AFF3CA
:1001B400008008BD000000006C000020D8910008F9
:1001C40081F0004102E000BF83F0004330B54FEA04
:1001D40041044FEA430594EA050F08BF90EA020F71
:1001E4001FBF54EA000C55EA020C7FEA645C7FEA04
:1001F400655C00F0E2804FEA5454D4EB5555B8BF27
:100204006D420CDD2C4480EA020281EA030382EA97
:10021400000083EA010180EA020281EA0303362D29
:1002240088BF30BD11F0004F4FEA01314FF4801CFC
:100234004CEA113102D0404261EB410113F0004F0E
:100244004FEA03334CEA133302D0524263EB4303C5
:1002540094EA050F00F0A780A4F10104D5F1200E63
:100264000DDB02FA0EFC22FA05F2801841F10001BE
:1002740003FA0EF2801843FA05F359410EE0A5F192
:1002840020050EF1200E012A03FA0EFC28BF4CF0C3
:10029400020C43FA05F3C01851EBE37101F0004579
:1002A40007D54FF0000EDCF1000C7EEB00006EEB86
:1002B4000101B1F5801F1BD3B1F5001F0CD3490810
:1002C4005FEA30004FEA3C0C04F101044FEA445267
:1002D40012F5800F80F09A80BCF1004F08BF5FEAEE
:1002E400500C50F1000041EB045141EA050130BDCE
:1002F4005FEA4C0C404141EB010111F4801FA4F171
:100304000104E9D191F0000F04BF01460020B1FAC5
:1003140081F308BF2033A3F10B03B3F120020CDAFD
:100324000C3208DD02F1140CC2F10C0201FA0CF0DB
:1003340021FA02F10CE002F11402D8BFC2F1200C40
:1003440001FA02F120FA0CFCDCBF41EA0C019040F6
:10035400E41AA2BF01EB0451294330BD6FEA04043F
:100364001F3C1CDA0C340EDC04F11404C4F120022A
:1003740020FA04F001FA02F340EA030021FA04F33C
:1003840045EA030130BDC4F10C04C4F1200220FA93
:1003940002F001FA04F340EA0300294630BD21FAD1
:1003A40004F0294630BD94F0000F83F4801306BF97
:1003B40081F480110134013D4EE77FEA645C18BF8B
:1003C4007FEA655C29D094EA050F08BF90EA020F22
:1003D40005D054EA000C04BF1946104630BD91EA1A
:1003E400030F1EBF0021002030BD5FEA545C05D11D
:1003F4004000494128BF41F0004130BD14F580045C
:100404003CBF01F5801130BD01F0004545F0FE41CF
:1004140041F470014FF0000030BD7FEA645C1ABF04
:10042400194610467FEA655C1CBF0B46024650EA3B
:10043400013406BF52EA033591EA030F41F4002167
:1004440030BD00BF90F0000F04BF0021704730B5ED
:100454004FF4806404F132044FF000054FF00001C2
:1004640050E700BF90F0000F04BF0021704730B583
:100474004FF4806404F1320410F0004548BF404258
:100484004FF000013EE700BF42004FEAE2014FEAAD
:1004940031014FEA02701FBF12F07F4393F07F4F88
:1004A40081F06051704792F0000F14BF93F07F4FBA
:1004B400704730B54FF4607401F0004521F00041FD
:1004C40020E700BF50EA010208BF704730B54FF083
:1004D40000050AE050EA010208BF704730B511F088
:1004E400004502D5404261EB41014FF4806404F1C0
:1004F40032045FEA915C3FF4DCAE4FF003025FEA42
:10050400DC0C18BF03325FEADC0C18BF033202EBC9
:10051400DC02C2F1200300FA03FC20FA02F001FA23
:1005240003FE40EA0E0021FA02F11444C1E600BFC2
:1005340080F0004002E000BF81F0004142001FBF94
:100544005FEA410392EA030F7FEA226C7FEA236C9D
:100554006AD04FEA1262D2EB1363C1BFD218414092
:1005640048404140B8BF5B42192B88BF704710F028
:10057400004F40F4000020F07F4018BF404211F0CB
:10058400004F41F4000121F07F4118BF494292EA33
:10059400030F3FD0A2F1010241FA03FC10EB0C005F
:1005A400C3F1200301FA03F100F0004302D54942EC
:1005B40060EB4000B0F5000F13D3B0F1807F06D399
:1005C40040084FEA310102F10102FE2A51D2B1F191
:1005D400004F40EBC25008BF20F0010040EA030086
:1005E4007047490040EB000010F4000FA2F1010233
:1005F400EDD1B0FA80FCACF1080CB2EB0C0200FABD
:100604000CF0AABF00EBC25052421843BCBFD0400A
:100614001843704792F0000F81F4000106BF80F484
:1006240000000132013BB5E74FEA41037FEA226C47
:1006340018BF7FEA236C21D092EA030F04D092F012
:10064400000F08BF0846704790EA010F1CBF002046
:10065400704712F07F4F04D1400028BF40F00040A3
:10066400704712F100723CBF00F50000704700F0C3
:10067400004343F0FE4040F4000070477FEA2262EA
:1006840016BF08467FEA23630146420206BF5FEABB
:10069400412390EA010F40F4800070474FF00003BB
:1006A40004E000BF10F0004348BF40425FEA000C82
:1006B40008BF704743F0964301464FF000001CE02A
:1006C40050EA010208BF70474FF000030AE000BF80
:1006D40050EA010208BF704711F0004302D54042BE
:1006E40061EB41015FEA010C02BF84460146002030
:1006F40043F0B64308BFA3F18053A3F50003BCFA4B
:100704008CF2083AA3EBC25310DB01FA02FC6344F7
:1007140000FA02FCC2F12002BCF1004F20FA02F2FE
:1007240043EB020008BF20F00100704702F12002F1
:1007340001FA02FCC2F1200250EA4C0021FA02F252
:1007440043EB020008BF20EADC7070474FF0FF3C27
:1007540006E000BF4FF0010C02E000BF4FF0010CB7
:100764004DF804CD4FEA40024FEA41037FEA226C80
:1007740018BF7FEA236C11D001B052EA530C18BFA2
:1007840090EA010F58BFB2EB030088BFC81738BF07
:100794006FEAE17018BF40F0010070477FEA226CF5
:1007A40002D15FEA402C05D17FEA236CE4D15FEAF1
:1007B400412CE1D05DF8040B704700BF8446084625
:1007C4006146FFE70FB5FFF7C9FF002848BF10F1E6
:1007D400000F0FBD4DF808EDFFF7F4FF0CBF01202B
:1007E40000205DF808FB00BF4DF808EDFFF7EAFFB5
:1007F40034BF012000205DF808FB00BF4DF808ED70
:10080400FFF7E0FF94BF012000205DF808FB00BF64
:100814004DF808EDFFF7D2FF94BF012000205DF8EA
:1008240008FB00BF4DF808EDFFF7C8FF34BF0120F7
:1008340000205DF808FB00BF42000ED2B2F1FE4F6B
:100844000BD34FF09E03B3EB126209D44FEA00239B
:1008540043F0004323FA02F070474FF00000704762
:1008640012F1610F01D1420202D14FF0FF30704703
:100874004FF00000704700BF53B94AB9002908BFC0
:1008840000281CBF4FF0FF314FF0FF3000F07AB961
:10089400ADF1080C6DE904CE00F006F8DDF804E0D3
:1008A400DDE9022304B070472DE9F0478C460E467B
:1008B4000446089D002B50D18A4217466CD9B2FADF
:1008C40082FEBEF1000F0BD0CEF1200C01FA0EF621
:1008D40020FA0CFC02FA0EF74CEA060C00FA0EF4AD
:1008E4003A0CBCFBF2F9BBB202FB19CC09FB03FACC
:1008F4004FEA144848EA0C46B2450AD9F61909F1F8
:10090400FF3180F02581B24540F22281A9F102092C
:100914003E44A6EB0A06B6FBF2F002FB106600FBAF
:1009240003F3A4B244EA0644A34209D9E41900F14A
:10093400FF3280F00B81A34240F2088102383C442C
:100944000021E41A40EA0940002D62D0002324FA71
:100954000EF42C606B60BDE8F0878B4207D9002D44
:1009640055D0002185E841000846BDE8F087B3FA78
:1009740083F1002940F08F80B34202D3824200F217
:10098400FC80841A66EB03060120B446002D40D097
:1009940085E81010BDE8F08712B90127B7FBF2F71C
:1009A400B7FA87FEBEF1000F35D10121F61B4FEADD
:1009B400174C1FFA87F8B6FBFCF20CFB126608FB17
:1009C40002F0230C43EA0646B04207D9F61902F1B5
:1009D400FF3302D2B04200F2D2801A46361AB6FB76
:1009E400FCF00CFB106608FB00F8A3B243EA0644D3
:1009F400A04507D9E41900F1FF3302D2A04500F263
:100A0400B9801846A4EB080440EA02409CE7294652
:100A14002846BDE8F08707FA0EF7CEF1200326FA40
:100A240003F24FEA174CB2FBFCF11FFA87F80CFBF8
:100A3400112206FA0EF620FA03F301FB08F93343F8
:100A44001E0C46EA0246B14500FA0EF409D9F6191D
:100A540001F1FF3280F08C80B14540F28980023987
:100A64003E44A6EB0906B6FBFCF00CFB106200FB4F
:100A740008F99EB246EA0246B14507D9F61900F1D3
:100A8400FF3371D2B1456FD902383E44A6EB090653
:100A940040EA01418FE7C1F1200722FA07F88B40B1
:100AA40048EA030326FA07F44FEA134EB4FBFEF9AF
:100AB4001FFA83FC0EFB19448E4020FA07F809FB49
:100AC4000CFA48EA06084FEA184646EA0444A245E6
:100AD40002FA01F200FA01F608D9E41809F1FF302C
:100AE40044D2A24542D9A9F102091C44A4EB0A0448
:100AF400B4FBFEF00EFB104400FB0CFC1FFA88F85C
:100B040048EA0444A44507D9E41800F1FF3E29D279
:100B1400A44527D902381C4440EA0940A0FB0289B5
:100B2400A4EB0C0CCC45C246CE4615D312D055B11D
:100B3400B6EB0A036CEB0E0606FA07F7CB401F432D
:100B4400CE402F606E600021BDE8F0871046F7E6C6
:100B54008946DEE64645EAD2B8EB020A69EB030EA3
:100B64000138E4E77046D7E718468FE78146BDE7CA
:100B7400114676E702383C4444E7084606E7023A61
:100B84003E442BE7704700BF084B10B50446186875
:100B94004FF47A73B0FBF3F000F094F8002221468E
:100BA4004FF0FF3000F04EF8002010BD0000002090
:100BB40008B50B4B03201A6842F400721A601A68D5
:100BC40042F480621A601A6842F480721A6000F07B
:100BD40027F80020FFF7D8FF06F0EEFE002008BD3E
:100BE400003C0240024A136801331360704700BF9F
:100BF4001C010020014B1868704700BF1C01002035
:100C040037B50190FFF7F6FF0546019C631C18BF3A
:100C14000134FFF7EFFF401BA042FAD303B030BD0D
:100C2400074A0002D36800F4E06023F4E0631B0485
:100C34001B0C43F0BF6343F400330343D36070479A
:100C440000ED00E0174B30B5DC68C4F30224C4F1B6
:100C54000703251D042B28BF0423062D4FF001058F
:100C640098BF002405FA03F303F1FF3388BF033C64
:100C74001940A14005FA04F4013C2240002842EA4C
:100C840001024FEA0212AFBF00F16040064B00F0D0
:100C94000F00D2B2A5BFD2B200F561401A5480F859
:100CA400002330BD00ED00E014ED00E00123420913
:100CB40000F01F0003FA00F0014B43F822007047D4
:100CC40000E100E00138B0F1807F0AD2F021064B48
:100CD400064A586082F823100020072298601A60A0
:100CE40070470120704700BF10E000E000ED00E015
:100CF40090F83530022B03D08023436501207047E0
:100D04000523026880F835301368002023F00103BE
:100D1400136070472DE9F04F0B6885B001930023F1
:100D2400DFF8B4816A4ADFF8B4914FF0010E019CF8
:100D34000EFA03FE0EEA0406B64540F0B2804C6893
:100D440024F01007022F16D14FF00F0C4FEAD30AEC
:100D540000EB8A0A03F0070BDAF820504FEA8B0BFA
:100D64000CFA0BFC25EA0C0C0D6905FA0BF545EAA7
:100D74000C05CAF8205003254FEA430A05FA0AF580
:100D8400ED43D0F800B004F0030C0BEA050B0CFAA9
:100D94000AFC013F4CEA0B0C012FC0F800C011D82B
:100DA400876807EA050BCF6807FA0AFC4CEA0B07C9
:100DB4008760476827EA0E0EC4F300179F4047EA8E
:100DC4000E074760C7683D408F6807FA0AF73D433E
:100DD400C560E50065D54FF0000B4FF00F0ECDF860
:100DE4000CB0D8F8447003F0030C47F48047C8F8FB
:100DF4004470D8F84470374D07F480470397039F35
:100E040023F0030707F1804707F59C37D7F808A0BC
:100E14004FEA8C0C0EFA0CFEA8422AEA0E0E47D0BA
:100E240005F58065A84245D005F58065A84243D004
:100E340005F58065A84241D005F58065A8423FD0FC
:100E440048453FD005F50065A8423DD005F58065CD
:100E5400A8423BD005F58065A84214BF09250825A2
:100E640005FA0CF545EA0E05BD60F743156814F460
:100E7400803F0CBF3D4035431560556814F4003F76
:100E84000CBF3D4035435560956814F4801F0CBF7A
:100E94003D4035439560D568A40254BF3D40354379
:100EA400D5600133102B7FF440AF05B0BDE8F08F5F
:100EB4005D46D5E70125D3E70225D1E70325CFE732
:100EC4000425CDE70525CBE70625C9E70725C7E7B0
:100ED400003C01400000024000380240001402407F
:100EE4000369194214BF0120002070470AB18161CF
:100EF40070470904FBE74369594041617047026840
:100F0400536913F480630DD06FF480635361042339
:100F1400202203640023036380F83C3080F83D20E2
:100F240001207047184670472DE9F84304461746D8
:100F34009946C1F307488EB22568B8F1010F0CBF7A
:100F44006B69AB6936EA030314BF0120002008B9BA
:100F5400BDE8F8836B695A0512D52B68202243F447
:100F640000732B606FF480636B610423236400239C
:100F74000120236384F83C3084F83D20BDE8F883E5
:100F84007B1CD9D04FB900232022236384F83C3042
:100F940084F83D200320BDE8F883FFF72BFEA0EB87
:100FA40009008742C8D2EEE72DE9F843044690468B
:100FB4001F46089EC1F307498DB22368B9F1010F9A
:100FC4000CBF5B699B6935EA03030CBF0123002353
:100FD400434502D00020BDE8F8837B1CEDD05FB907
:100FE40000232022236384F83C3084F83D2003202E
:100FF40084F83E30BDE8F883FFF7FCFD801B874290
:10100400DBD2EDE770B504460D46164623685B69EE
:101014001B0601D5002070BD2046FFF770FFA8B95C
:101024006A1CF3D065B9236C202243F020032364A7
:1010340000230320236384F83C3084F83D2070BDF2
:10104400FFF7D8FD801B8542E0D2ECE7012070BD9C
:101054002DE9FF4115460268984613680B9E43F438
:10106400807313600F4600960A9B00224FF0011113
:101074000446FFF799FF68B9236807F0FE071F616C
:101084000A9A33461A492046FFF74EFF30B1236CC3
:10109400042B18D0032004B0BDE8F081236803902A
:1010A4005A690A9903929B69324603932046039B2B
:1010B400FFF7A8FF48B1236C042BEBD12268136817
:1010C40043F4007313600120E5E7B8F1010F2368CE
:1010D40002D1EDB21D61DEE72A0A1A610A9932468D
:1010E4002046FFF78FFF0028E5D12368F1E700BF12
:1010F400020001002DE9FF419846036816461A686C
:101104000B9D42F480621A601A680F4642F48072A2
:101114001A604FF0011100950A9B00220446FFF764
:1011240043FF80B92368FFB207F0FE021A612D491C
:101134002B460A9A2046FFF7F7FE40B1236C042B96
:1011440001D1012000E0032004B0BDE8F081236850
:1011540003905A690A9903929B692A46039320468D
:10116400039BFFF74FFF40B1236C042BEBD12268A4
:10117400136843F400731360E3E7B8F1010F2368C5
:1011840024D1F6B21E612A460A992046FFF73AFF97
:1011940002460028E8D1216820460B6843F4807396
:1011A4000B6000950A9B4FF00111FFF7FDFE00282C
:1011B400C9D1236847F001071F610A9A2B460949E0
:1011C4002046FFF7B1FE0028B8D1BDE7320A1A6104
:1011D4000A992A462046FFF715FF0028C4D1236840
:1011E400CFE700BF0200010070B504460D46164665
:1011F4002068436913F0400301D0002070BD4269A8
:10120400D2060BD56FF0100242612022236484F8C9
:101214003C302363012084F83D2070BD5DB9236C0C
:10122400032043F020032364202384F83D3000236B
:1012340084F83C3070BDFFF7DDFC801B8542D7D2BB
:10124400EDE770B504460D46164623685B695B07F7
:1012540001D5002070BD2046FFF751FEA8B96A1CD5
:10126400F3D065B9236C202243F0200323640023C8
:101274000320236384F83C3084F83D2070BDFFF7DD
:10128400B9FC801B8542E0D2ECE7012070BD000070
:1012940070B50446002863D090F83D3003F0FF0297
:1012A4001BB980F83C2006F0A3FB2423226884F8B1
:1012B4003D3013682B4E23F00103136000F038FC1B
:1012C4006368294DB342B0FBF5F588BF4FF49671BE
:1012D400226888BF6943556085BF4FF47A75B1FBB6
:1012E400F5F1691C0131B342116221D85B00B0FBF6
:1012F400F3F0C0F30B03032B98BF0420216AE369C6
:10130400D0610B431360E168236900200B439360B1
:10131400A16963690B43D360136843F0010313604D
:101324002023206484F83D30206384F83E0070BD9F
:10133400A16849B903EB4303B0FBF3F0C0F30B031B
:1013440063B140F40040D9E719214B43B0FBF3F0FB
:10135400C0F30B0313B140F44040CFE70120CDE7C5
:10136400012070BDA086010040420F002DE9F34723
:1013740004469A46884691460C9EFFF73BFC94F837
:101384003D300546202B03D0022002B0BDE8F08793
:101394000090192301223E492046FFF705FE00284C
:1013A400F2D194F83C30012BEED0012384F83C3088
:1013B400236800271A684146D20758BF1A68204696
:1013C4005CBF42F001021A601A6822F400621A60DB
:1013D400212384F83D30402384F83E300A9B27645F
:1013E4006362BDF82C30019563852A4B0096E36255
:1013F400638D4A4623855346FFF72AFE00282AD0E8
:10140400236C84F83C70042B07D10120BDE7FFF75F
:10141400F9FD20B1236C042B34D00320B5E7616AB5
:1014240027684B1C63620B78228D3B61638D501ED1
:10143400013B9BB263857B6980B25B0720850AD53B
:1014440048B18B1C63624B78023A3B61638D228501
:10145400013B9BB26385238D2A4631462046002BEF
:10146400D5D1FFF7EEFE0028D4D12268136843F4E7
:1014740000731360202384F83C0084F83D3084F822
:101484003E0082E72268136843F400731360BCE7EC
:10149400020010000000FFFF2DE9F047044686B06B
:1014A4009A460D469146109FFFF7A4FB94F83D30F1
:1014B4000646202B04D00225284606B0BDE8F08756
:1014C4000090192301227A492046FFF76DFD002878
:1014D400F1D194F83C30012BEDD0012384F83C3059
:1014E40023684FF000081A682946D20758BF1A68C3
:1014F40020465CBF42F001021A601A6822F40062BE
:101504001A60222384F83D30402384F83E300E9B39
:10151400C4F840806362BDF83C3001966385654B36
:101524000097E362638D4A4623855346FFF7E2FD45
:10153400054630B1236C84F83C80042B3AD1012554
:10154400BAE7228D236892B902905A6902929A6985
:101554000292029A1A6842F400721A60202384F8F4
:101564003D30002384F83E3084F83C30A4E7012A5F
:1015740022D11A6822F480621A6003905A69039295
:101584009A690392039A1A6842F400721A60DFF8A7
:101594002881238D002BE1D0032B6BD8012B23D181
:1015A400324639462046FFF71FFE002839D0236C07
:1015B400202BC4D103257FE7022A0ED11A6822F416
:1015C40080621A601A6842F400621A6004905A69D0
:1015D40004929B690493049BD9E705905A69059288
:1015E4009B690593059BD2E7022B00963B464FF07F
:1015F40000024146204622D1FFF7D6FC0028D9D16B
:1016040023681A6842F400721A60626A1B69511CEA
:1016140061621370238D013B2385638D013B9BB273
:101624006385636A5A1C6262226812691A70238D88
:10163400013B2385638D013B9BB26385A9E7FFF7DB
:10164400B3FC02460028B5D12368196821F48061EF
:101654001960616A1B69481C60620B70238D0096D7
:10166400013B2385638D4146013B9BB26385204644
:101674003B46C1E7324639462046FFF7B5FD002810
:1016840095D1636A5A1C6262226812691A70238DAA
:101694002268013B2385638D013B9BB263855369BB
:1016A4005B077FF576AF636A591C6162BDE700BFD3
:1016B400020010000000FFFF04000100F7B504461B
:1016C40010B9012003B0F0BD0368D80738D42368EB
:1016D40099076BD423681E0700F1B88023685D075F
:1016E40028D500230193A54BA54D1A6C42F08052D6
:1016F4001A641B6C03F080530193019B2B6843F421
:1017040080732B60FFF776FA06462B68DA0540F102
:10171400BF809C4B227A1A70A368002B00F0C6800D
:10172400FFF768FA41F288370646944D2B6F9B0702
:1017340040F1B580A269002A40F0C8800020C1E7CA
:101744008E4B9A6802F00C02042A07D09A6802F0C1
:101754000C02082A0AD15B685A0207D5874B1B681A
:101764009B03B4D56368002BB1D1AAE7864B2279D9
:101774001A7063686BB1FFF73DFA06467F4D2B681C
:101784009F03A4D4FFF736FA801B6428F7D90320FB
:1017940098E7FFF72FFA0646784D2B68980396D5FD
:1017A400FFF728FA801B6428F7D9F0E7734B9A688F
:1017B40012F00C0F07D09A6802F00C02082A17D115
:1017C4005B68590214D46D4B1A68920703D5E2681A
:1017D400012A7FF476AF1868F82292FAA2F2B2FADC
:1017E40082F122698A4020F0F8010A431A6071E705
:1017F400E268664BDAB101221A60FFF7FBF906468C
:101804005E4D2B689B070CD52968F82393FAA3F344
:10181400B3FA83F22369934021F0F80213432B6057
:1018240058E7FFF7E7F9801B0228EAD9AFE71A6007
:10183400FFF7E0F90646514D2B689F077FF54AAF45
:10184400FFF7D8F9801B0228F6D9A0E76269504B4C
:101854007AB101221A60FFF7CDF90646474D6B6F46
:1018640098073FF53BAFFFF7C5F9801B0228F6D96F
:101874008DE71A60FFF7BEF90646404D6B6F990776
:101884007FF52CAFFFF7B6F9801B0228F6D97EE767
:10189400FFF7B0F9801B02287FF637AF77E7FFF731
:1018A400A9F9801BB8427FF641AF70E7FFF7A2F9B0
:1018B40041F288370646314D2B6F98077FF53AAFD2
:1018C400FFF798F9801BB842F6D960E72B4DAB6857
:1018D40003F00C03082B3FF4F4AE00232D4E022A30
:1018E40033603ED1FFF786F907462B68990132D45D
:1018F40047F6C07797FAA7F74FF44032B7FA87F75D
:1019040092FAA2F24FF07061B2FA82F091FAA1F168
:10191400B1FA81F1226AE3691343626A02FA07F7B2
:10192400A26A3B435208013A82401343E26A134CD1
:1019340002FA01F10B436B6001233360FFF75AF99C
:10194400054623689A013FF5F9AEFFF753F9401BAA
:101954006428F6D91BE7FFF74DF9C01B6428C4D9E6
:1019640015E7FFF747F904462B689B017FF5E6AEC0
:10197400FFF740F9001B6428F6D908E70038024055
:1019840000700040703802400238024000004742B4
:10199400800E474260004742134908B58B6803F044
:1019A4000C03042B03D0082B03D0104808BD1048A7
:1019B40008BD4A684B68496813F4800314BF0C4897
:1019C4000A48C1F3881118BF002302F03F02A1FBAB
:1019D4000001FEF751FF044B5B68C3F3014301337D
:1019E4005B00B0FBF3F008BD003802400024F400B3
:1019F40040787D012DE9F0410D46044610B90120DF
:101A0400BDE8F081464B1A6802F00F028A422ED3D9
:101A140021688F0733D4C80746D4414B1A6802F0B3
:101A24000F0295426AD32268510770D4130707D571
:101A34003C4A2169936823F4604343EAC1039360F9
:101A4400FFF7AAFF374BF0229B6892FAA2F2B2FA90
:101A540082F203F0F003D340334AD35CD840334BD3
:101A640018600020FFF790F80020BDE8F081CAB2AA
:101A74001A701B6803F00F039942C0D1C8E7294BC1
:101A840011F0040F1EBF9A6842F4E0529A600E07E8
:101A940042BF9A6842F460429A609A68A06822F051
:101AA400F00202439A60B6E761681E4B01291A6886
:101AB4001CD112F4003FA2D09A6841F2883822F077
:101AC40003020A439A60FFF795F80746154EB36878
:101AD400626803F00C03B3EB820F9ED0FFF78AF821
:101AE400C01B4045F3D90320BDE8F081022902D18F
:101AF40012F0007FDFE712F0020FDCE7EAB21A709F
:101B04001B6803F00F039D427FF479AF8BE705490F
:101B1400E0688B6823F4E05303438B6086E700BFDF
:101B2400003C024000380240B2930008000000204C
:101B3400084B4FF4E0529B6892FAA2F2B2FA82F296
:101B440003F4E053D340044AD35C044A1068D840F9
:101B5400704700BF00380240C29300080000002014
:101B6400084B4FF460429B6892FAA2F2B2FA82F2F6
:101B740003F46043D340044AD35C044A1068D84059
:101B8400704700BF00380240C293000800000020E4
:101B940003680020DA6842F00102DA601A6842F051
:101BA40001021A60704770477047704770470368B6
:101BB40010B51A69044691070ED5DA6892070BD559
:101BC4006FF002021A6101229B6902779B0777D0AA
:101BD400FFF7EAFF0023237723681A69500710D51B
:101BE400DA6851070DD56FF004021A6102229B696D
:101BF400227713F4407F204668D0FFF7D5FF0023F7
:101C0400237723681A6912070FD5DA6810070CD5F1
:101C14006FF008021A610422DB69227799072046D3
:101C24005AD0FFF7C1FF0023237723681A69D2062D
:101C340010D5DA68D0060DD56FF010021A610822AB
:101C4400DB69227713F4407F20464BD0FFF7ACFFCB
:101C54000023237723681A69D10708D5DA68D207E5
:101C640005D56FF0010220461A6105F09DFB23683B
:101C74001A69100608D5DA68110605D56FF08002D6
:101C840020461A6100F0DBF823681A69520608D569
:101C9400DA68500605D56FF0400220461A61FFF756
:101CA40085FF23681A69910622D5DA6892061FD542
:101CB4006FF020022046BDE810401A6100F0BEB863
:101CC400FFF771FF2046FFF770FF83E7FFF76BFF15
:101CD4002046FFF76AFF92E7FFF765FF2046FFF70C
:101CE40064FFA0E7FFF75FFF2046FFF75EFFAFE763
:101CF40010BD0000304A0368904212D0B0F1804F0A
:101D04000FD0A2F57C4290420BD002F58062904243
:101D140007D002F58062904203D002F578429042E7
:101D24001DD14A6823F070031343234A904204D11F
:101D3400CA6823F44073134328E0B0F1804FF7D00E
:101D44001E4A9042F4D002F580629042F0D002F52F
:101D540080629042ECD002F578429042E8D0184A72
:101D64009042E5D002F580629042E1D002F58062B3
:101D74009042DDD0A2F598329042D9D002F580622B
:101D84009042D5D002F580629042D1D04A6923F0C6
:101D94008003134303608B68C3620B688362064B42
:101DA400984206D003F58063984202D00123436130
:101DB40070470B690363F9E7000001400004004029
:101DC4000040014010B50446A0B190F83D3003F046
:101DD400FF021BB980F83C2005F062FE0223206854
:101DE40084F83D30211DFFF785FF0123002084F88E
:101DF4003D3010BD012010BD90F83C3010B5012BD2
:101E04004FF0020318D080F83D3003680C685A681C
:101E1400496822F070025A605A6822435A609A68EC
:101E240022F080029A609A680A439A60012380F83B
:101E34003D30002380F83C30184610BD7047704791
:101E44000368DA6822F49072DA605A6922F00102B7
:101E54005A61202380F83A30704700002DE9F0479A
:101E640004460668C2683369C16923F440531343C6
:101E7400336183680069F2680343606922F416429F
:101E8400034322F00C020B431343F3607369A2690A
:101E940023F440731343B1F5004F73617A4B7CD143
:101EA4009E4203D003F580639E4244D1FFF758FE5F
:101EB400192505FB00F360684FF064094000B3FB8B
:101EC400F0F3B3FBF9F34FEA0318FFF749FE684355
:101ED40063685B00B0FBF3F7FFF742FE6843636897
:101EE4005B00B0FBF3F3B3FBF9F309FB1373DB0003
:101EF4003233B3FBF9F35B0003F4F877FFF730FEFA
:101F0400684362685200B0FBF2FAFFF729FE6843A7
:101F140063685B00B0FBF3F3B3FBF9F309FB13A3B2
:101F2400DB003233B3FBF9F303F0070343443B44D0
:101F3400B360BDE8F087FFF7FBFD192505FB00F34F
:101F440060684FF064094000B3FBF0F3B3FBF9F3AE
:101F54004FEA0318FFF7ECFD684363685B00B0FBCE
:101F6400F3F7FFF7E5FD684363685B00B0FBF3F349
:101F7400B3FBF9F309FB1373DB003233B3FBF9F35F
:101F84005B0003F4F877FFF7D3FD684362685200FF
:101F9400B0FBF2FAFFF7CCFDB9E79E4202D03B4B0F
:101FA4009E4240D1FFF7DCFD192505FB00F367686D
:101FB4004FF06409BF00B3FBF7F3B3FBF9F31F0160
:101FC400FFF7CEFD684363689B00B0FBF3F8FFF7AF
:101FD400C7FD684363689B00B0FBF3F3B3FBF9F3FD
:101FE40009FB13831B013233B3FBF9F303F0F0084D
:101FF400FFF7B6FD684362689200B0FBF2FAFFF7A0
:10200400AFFD684363689B00B0FBF3F3B3FBF9F3E4
:1020140009FB13A31B013233B3FBF9F303F00F03E2
:1020240043EA080383E7FFF783FD192505FB00F363
:1020340067684FF06409BF00B3FBF7F3B3FBF9F330
:102044001F01FFF775FD684363689B00B0FBF3F85D
:10205400FFF76EFD684363689B00B0FBF3F3B3FBCB
:10206400F9F309FB13831B013233B3FBF9F303F0D8
:10207400F008FFF75DFD684362689200B0FBF2FA76
:10208400FFF756FDBDE700BF0010014000140140FA
:10209400F8B504460E4617461D4621680B6836EA15
:1020A400030301D10020F8BD6B1CF7D095B9236858
:1020B4000320DA6822F4D072DA605A6922F001024D
:1020C4005A61202384F8393084F83A30002384F8A4
:1020D4003830F8BDFEF78EFDC01B8542DDD2E6E741
:1020E40010B5044640B390F8393003F0FF021BB931
:1020F40080F8382005F0ECFC2423226884F8393079
:10210400D368204623F40053D360FFF7A7FE236867
:1021140000201A6922F490421A615A6922F02A02B4
:102124005A61DA6842F40052DA602023E06384F8EA
:10213400393084F83A3010BD012010BD2DE9F0414A
:102144001F4690F839300446202B0D4690464ED158
:10215400002949D0002A47D090F83830012B46D0C6
:10216400012380F838300023C363212380F83930F9
:10217400FEF740FD0646A4F82480A4F82680E38CEC
:102184009BB26BB93B46324640212046FFF780FFA5
:10219400A8B9202384F8380084F83930BDE8F081E8
:1021A400E38C3246013B9BB2E384A3688021B3F500
:1021B400805F20463B460ED1FFF76AFF10B1032033
:1021C400BDE8F0812B882268C3F3080353602369B8
:1021D40043B90235D3E7FFF75BFF0028EFD123684B
:1021E4002A785A600135CAE70120BDE8F08102204F
:1021F400BDE8F08190F83A30202B1CD1C9B1C2B1AE
:1022040090F83830012B16D0C28582850023222213
:10221400C36380F83A2002688162516980F83830DB
:1022240041F001015161D168184641F49071D160C7
:1022340070470120704702207047704790F83A3089
:1022440010B5222B32D183680169B3F5805F02682F
:10225400836A1FD15268C9B9C2F3080223F8022B5A
:102264008362C48D013CA4B2C4856CB90368DA6886
:1022740022F49072DA605A6922F001025A61202332
:1022840080F83A3005F0B4F8002010BDD2B223F83B
:10229400012BE5E721B9591C526881621A70E0E705
:1022A4005268591C816202F07F02F7E7022010BDD8
:1022B40070470000036870B51A6804461607D968A9
:1022C4005D6907D196065AD58D0658D5BDE870408C
:1022D400FFF7B4BF15F0010502D111F4907F4ED081
:1022E400D30705D5CE0542BFE36B43F00103E36397
:1022F400500704D51DB1E36B43F00203E363930776
:1023040004D51DB1E36B43F00403E363160704D55E
:102314001DB1E36B43F00803E363E36B002B66D06A
:10232400950604D5880602D52046FFF787FF236863
:1023340020465D69E26B110702D415F040051AD0FE
:10234400FFF77EFD23685A69520610D55A69606BFF
:1023540022F040025A6150B1254B0365FEF7C8FCD8
:10236400002844D0606BBDE87040036D18472046D8
:10237400FFF79EFF70BDFFF79BFFE56370BD160678
:1023840027D50D0625D594F83920212A2FD1A26806
:10239400B2F5805F226A17D11188C1F30801596030
:1023A400216979B902322262E28C013A92B2E28462
:1023B400EAB9DA6822F08002DA60DA6842F04002B0
:1023C400DA6070BD0132EEE7511C216212785A6066
:1023D400EAE750060BD54A0609D5DA68204622F00A
:1023E4004002DA60202384F83930FFF726FF70BDFD
:1023F400F923000808B50023806BC385C384FFF765
:1024040057FF08BD014B1870704700BFBC00002087
:10241400014B1878704700BFBC00002010B504467B
:10242400087801F061FA206010BD38B504460878D8
:102434000D4601F059FA2060687801F055FA01461A
:102444002068FEF77BF82060A87801F04DFA014679
:102454002068FEF773F82060E87801F045FA014639
:102464002068FEF76BF8206038BD38B5044608785C
:102474000D4601F0C9FA2060687801F0C5FA0146FA
:102484002068FEF75BF82060A87801F075FA014631
:102494002068FEF753F8206038BD00000138122888
:1024A40038D8DFE800F00A3737372237370E1215ED
:1024B400191C1F25282B2E31340017491748FFF704
:1024C400ADBF17491748FFF7B0BF17491748FAE7D8
:1024D40017491848FFF7C9BF17491848FAE71849B8
:1024E4001848F7E718491948F4E719491948E6E77D
:1024F40019491A48E7E71A491A48E4E71A491B48F0
:10250400E8E71B491B48E5E71B491C48E2E71C496F
:102514001C48DFE7704700BFA607002084000020A6
:10252400A707002098000020AB0700209C00002093
:10253400AF07002088000020B20700208C00002094
:10254400B507002090000020B80700209400002068
:10255400BB070020A0000020BC070020B40000201E
:10256400C0070020B8000020C4070020A4000020F9
:10257400C7070020A8000020CA070020AC000020E4
:10258400CD070020B00000200023DAB2815C0133C3
:102594000029FAD1104670472DE9F0474FF0100A90
:1025A4004FF020099EB001AF80460D46144600212D
:1025B4005246384605AE05F018FC4A46002130461E
:1025C40005F013FC4FF48053ADF834304FF400633E
:1025D400ADF836304FF40053ADF838304FF4804343
:1025E400ADF83C304FF40043ADF83E300423ADF871
:1025F40040300823ADF842304023ADF84830802302
:10260400ADF846A0ADF84490ADF84A30B8F1000FEB
:1026140002D0404600F01BFA00224FF478413B48B8
:10262400FEF764FC0022FC213948FEF75FFC002D14
:1026340067D12A464FF400613448FEF757FC0FABCC
:1026440093E8030016AB87E8030093E80300012234
:1026540086E803004FF400512C48FEF747FC14F0C1
:10266400010218BF01224FF480412848FEF73EFCC6
:1026740014F0020218BF01224FF400412348FEF770
:1026840035FC14F0040218BF012204212048FEF78F
:102694002DFC14F0080218BF012208211C48FEF783
:1026A40025FC14F0100218BF012220211848FEF75F
:1026B4001DFC14F0200218BF012210211448FEF75B
:1026C40015FC14F0400218BF012240211048FEF707
:1026D4000DFC23064CBF0122002280210C48FEF78A
:1026E40005FC00224FF400510848FEF7FFFB55B9E2
:1026F40001224FF4006105481EB0BDE8F047FEF723
:10270400F5BB012296E70022F3E700BF000C02406C
:1027140000180240002138B5AF4C0C220846FFF7E0
:102724003BFFA07901F0E0F8AC4BAD4D1860E079C7
:1027340001F0DAF801462868FDF700FF2860207AE6
:1027440001F0D2F801462868FDF7F8FE2860607AA7
:1027540001F0CAF801462868FDF7F0FE2860A07A67
:1027640001F0C2F801462868FDF7E8FE2860E07A27
:1027740001F0BAF89B4D01462868FDF7DFFE28609A
:10278400207B01F0B1F801462868FDF7D7FE2860E8
:10279400607B01F0A9F801462868FDF7CFFE2860A8
:1027A400A07B01F0A1F801462868FDF7C7FE286068
:1027B400E07B01F029F98C4D01462868FDF7BEFE47
:1027C4002860207C01F020F901462868FDF7B6FE58
:1027D4002860607C01F0D0F801462868FDF7AEFE61
:1027E4002860A07C01F010F9804D01462868FDF7AF
:1027F400A5FE2860E07C01F007F901462868FDF792
:102804009DFE2860207D01F0B7F801462868FDF799
:1028140095FE2860607D01F0F7F8754D0146286843
:10282400FDF78CFE2860A07D01F0EEF801462868D3
:10283400FDF784FE2860E07D01F09EF801462868DB
:10284400FDF77CFE2860207E01F0DEF8694D01462C
:102854002868FDF773FE2860607E01F0D5F8014614
:102864002868FDF76BFE2860A07E01F085F801461C
:102874002868FDF763FE2860E07E01F035F85E4BC2
:102884005E4D1860207F01F02FF801462868FDF79F
:1028940055FE2860607F01F027F801462868FDF79F
:1028A4004DFE2860A07F01F01FF801462868FDF75F
:1028B40045FE2860E07F01F017F801462868FDF71F
:1028C4003DFE286094F8200001F00EF84C4D0146BE
:1028D4002868FDF733FE286094F8210001F004F81D
:1028E40001462868FDF72AFE286094F8220000F0CB
:1028F400FBFF01462868FDF721FE286094F82300B9
:1029040000F0F2FF01462868FDF718FE286094F8ED
:10291400240001F079F83B4D01462868FDF70EFECE
:10292400286094F8250001F06FF801462868FDF747
:1029340005FE286094F8260001F01EF80146286878
:10294400FDF7FCFD286094F8270001F05DF82E4D9A
:1029540001462868FDF7F2FD286094F8280001F08C
:1029640053F801462868FDF7E9FD286094F829002A
:1029740001F002F801462868FDF7E0FD286094F8AC
:102984002A0001F041F8214D01462868FDF7D6FDE3
:10299400286094F82B0001F037F801462868FDF709
:1029A400CDFD286094F82C0000F0E6FF014628686D
:1029B400FDF7C4FD286094F82D0001F025F8144DAE
:1029C40001462868FDF7BAFD286094F82E0001F04E
:1029D4001BF801461EE000BFA00700208400002071
:1029E400980000209C000020880000208C0000201B
:1029F4009000002094000020A0000020B4000020DB
:102A0400B8000020A4000020A8000020AC00002092
:102A1400B00000202868FDF791FD286094F82F008D
:102A240000F0AAFF01462868FDF788FD286038BD3C
:102A340000210F220846FFF7AFBD00210C220846F3
:102A4400FFF7AABD002101220846FFF7A5BD00211A
:102A540001280CBF8022C0220846FFF79DBD00005C
:102A64002DE9F04F10252024A1B00DF10C0A904659
:102A740007462A468946504600210DF11C0B05F0F5
:102A8400B4F922460021584605F0AFF94FF48053BB
:102A9400ADF83C304FF40063ADF83E304FF40053D2
:102AA400ADF840304FF48043ADF844304FF4004368
:102AB400ADF846300423ADF848300823ADF84A3069
:102AC4004023ADF8503080234046ADF84E50ADF869
:102AD4004C40ADF85230FFF757FD4646504D514C2F
:102AE4000190A6EB0803019ADBB29A4202D821B006
:102AF400BDE8F08F002F40F08780002700224FF4BC
:102B040078412846FEF7F2F90022FC212046FEF720
:102B1400EDF9B9F1000F7ED14A464FF40061284621
:102B2400FEF7E4F911AB93E8030018AB8AE803005D
:102B340093E8030001228BE803004FF40051284678
:102B4400FEF7D4F916F8012B4FF4804112F001027C
:102B540018BF01222846FEF7C9F916F8012C4FF4D4
:102B6400004112F0020218BF01222846FEF7BEF906
:102B740016F8012C042112F0040218BF0122204689
:102B8400FEF7B4F916F8012C082112F0080218BF58
:102B940001222046FEF7AAF916F8012C202112F092
:102BA400100218BF01222046FEF7A0F916F8012CE6
:102BB400102112F0200218BF01222046FEF796F9D8
:102BC40016F8012C402112F0400218BF01222046C1
:102BD400FEF78CF916F9013C8021002BB4BF0122C9
:102BE40000222046FEF782F900224FF400512846C5
:102BF400FEF77CF9B9F1000F0FD101224FF4006107
:102C04002846FEF773F96CE73846FFF720FF022FDA
:102C14003FF473AF72E701227FE70022EEE700BFC3
:102C2400000C024000180240014B1878704700BFA6
:102C3400BE0000201FB5102400212246684605F07E
:102C4400D4F8FFF7FAFEFFF7FDFE0C4A012100203D
:102C5400FFF706FF224601210020FFF79DFC0849EB
:102C6400684605F021FA6A4601210220FFF7F8FEC2
:102C74000022044B1A7004B010BD00BFB4920008C7
:102C8400C4920008BE0000201FB510240021224673
:102C9400684605F0AAF8FFF7D0FEFFF7D3FE0F4A07
:102CA40001210020FFF7DCFE224601210020FFF76E
:102CB40073FC0B4B1868FDF7E7FB0B46024609490A
:102CC400684605F0CDF96A4601210220FFF7C8FEE7
:102CD4000122054B1A7004B010BD00BF8992000890
:102CE4008400002098920008BE0000201FB5102424
:102CF40000212246684605F078F8FFF79EFEFFF7AC
:102D0400A1FE112201210020FFF746FC0E4A0121F9
:102D14000020FFF7A5FE224601210020FFF73CFC1E
:102D24000A4B1868FDF7B0FB0B4602460849684693
:102D340005F096F96A4601210220FFF791FE02226E
:102D4400044B1A7004B010BDD09200089800002003
:102D540098920008BE0000201FB51022002168468A
:102D640005F043F8FFF769FEFFF76CFE112201211D
:102D74000020FFF711FC0D4A01210020FFF770FE2F
:102D84000B4B1868FDF780FB0B4602460949684661
:102D940005F066F96A4601210220FFF761FE03226D
:102DA400054B1A7005B05DF804FB00BFA89200083B
:102DB4008800002098920008BE0000201FB5102251
:102DC4000021684605F011F8FFF737FEFFF73AFED9
:102DD400112201210020FFF7DFFB0A4A0121002014
:102DE400FFF73EFE0849684605F05EF96A46012190
:102DF4000220FFF735FE0422044B1A7005B05DF87B
:102E040004FB00BFFA920008C4920008BE00002030
:102E14001FB5102400212246684604F0E6FFFFF7A0
:102E24000CFEFFF70FFE0F4A01210020FFF718FEEA
:102E3400224601210020FFF7AFFB0B4B1868FDF77A
:102E440023FB0B4602460949684605F009F96A4620
:102E540001210220FFF704FE0522054B1A7004B07D
:102E640010BD00BFDF920008A00000209892000867
:102E7400BE0000201FB5102400212246684604F03D
:102E8400B4FFFFF7DAFDFFF7DDFD11220121002079
:102E9400FFF782FB0E4A01210020FFF7E1FD2246E5
:102EA40001210020FFF778FB0A4B1868FDF7ECFAC4
:102EB4000B4602460849684605F0D2F86A460121E5
:102EC4000220FFF7CDFD0622044B1A7004B010BD9A
:102ED40006930008B400002098920008BE00002069
:102EE4001FB510220021684604F07FFFFFF7A5FDFF
:102EF400FFF7A8FD112201210020FFF74DFB0D4A29
:102F040001210020FFF7ACFD0B4B1868FDF7BCFA5C
:102F14000B4602460949684605F0A2F86A460121B3
:102F24000220FFF79DFD0722054B1A7005B05DF8DE
:102F340004FB00BFEE920008A40000209892000851
:102F4400BE0000202DE9F0410C46164686B0102242
:102F54000021804602A804F048FFFFF769FD2168BC
:102F64003046FDF7EBFA194F206039460546FDF768
:102F740059FC18B1276006B0BDE8F0810027284647
:102F84003946FDF731FC0028F4D12846FDF77CFAD8
:102F940002460B4602A80E4905F062F82068FDF7C8
:102FA40073FA044630460D46FDF76EFA2B46CDE91A
:102FB40000012246074804F021FF02AA0121022051
:102FC400FFF74EFD044B83F80080D4E70000F04186
:102FD4009892000811920008BE000020F0B50C463B
:102FE400154685B0102200210746684604F0FDFE10
:102FF400FFF71EFD21682846FDF7A0FA104E206059
:1030040031460546FDF70EFC10B1266005B0F0BD53
:10301400002628463146FDF7E7FB0028F5D128466F
:10302400FDF732FA0B4602460649684605F018F8E1
:103034006A4601210220FFF713FD034B1F70E5E7E9
:103044000000F04298920008BE000020F0B50C4643
:10305400154685B0102200210746684604F0C5FED7
:10306400FFF7E6FC21682846FDF768FA104E206059
:1030740031460546FDF7D6FB10B1266005B0F0BD1C
:10308400002628463146FDF7AFFB0028F5D1284637
:10309400FDF7FAF90B4602460649684604F0E0FFDC
:1030A4006A4601210220FFF7DBFC034B1F70E5E7B2
:1030B4000000B44298920008BE00002030B50446D7
:1030C40085B010220D466846002104F08EFEFFF7FD
:1030D400B4FCFFF7B7FC082C01D00E2C1BD1154A09
:1030E40001210020FFF7BCFC102201210020FFF782
:1030F40053FA2868FDF7C8F90B4602460E4968469C
:1031040004F0AEFF6A4601210220FFF7A9FC0B4B35
:103114001C7005B030BD092C01D00F2CE9D111224F
:1031240001210020FFF738FA054A01210020FFF7AA
:1031340097FCDEE76992000898920008BE00002020
:103144007992000830B5044685B010220D466846D1
:10315400002104F04AFEFFF770FCFFF773FC0A2C11
:1031640001D0102C1BD1204A01210020FFF778FC4C
:10317400102201210020FFF70FFA2868FDF784F9D7
:103184000B4602461949684604F06AFF6A46012163
:103194000220FFF765FC164B1C7005B030BD0B2CEC
:1031A40001D0112C06D1112201210020FFF7F4F9DE
:1031B400104AD9E70C2C01D0122C06D1112201217E
:1031C4000020FFF7E9F90C4ACEE70D2C01D0132CAF
:1031D400D3D1112201210020FFF7DEF9074A012192
:1031E4000020FFF73DFCC8E72C92000898920008E5
:1031F400BE0000203C9200084B9200085A9200083E
:1032040038B5AD4D04462B789BB968B9FFF71AFC65
:103214002046AA4A0121FFF723FCBDE83840A84A0A
:1032240001210220FFF71CBCFFF704FD01232B70D2
:1032340038BD022803D1BDE83840FFF7FBBCA14BE1
:103244001D782846FFF72AF9212D00F27081DFE866
:1032540015F022003800450058002F00620071006C
:103264007E00850093009E00AC00B900C600CE002D
:10327400DD00E500F000FD000A0112012D016F01DF
:103284008701B301DD0108023302480261027A02B8
:10329400A502EA021503042C03D1BDE83840FFF768
:1032A4008DBD052C40F04381BDE83840FFF7ECBCF0
:1032B400032CC0D0052C40F03A81BDE83840FFF71C
:1032C400A7BD042C03D1BDE83840FFF70FBD052C82
:1032D40040F02D8100227C49142027E0042C03D1E6
:1032E400BDE83840FFF738BD032CDDD0052C05D1EF
:1032F40008207649BDE83840FFF7E0BE012C9AD09B
:1033040038BD032CDFD0052CF8D10A207049BDE864
:103314003840FFF717BF042C03D1BDE83840FFF74E
:10332400A9BD052CEAD100221B206A49BDE838401A
:10333400FFF708BE042C03D1BDE83840FFF7D0BD29
:10334400032CBAD0052CD9D163490E20D2E7032C23
:10335400E3D0052CD2D161491020D8E7042C02D146
:103364005F490920C6E7052C03D1002257491520DF
:1033740009E0012C98D038BD032CB9D0052CF8D124
:10338400002216205649BDE83840FFF727BE042C1A
:1033940002D154490B20BAE7052CEAD100224C494A
:1033A4001720BDE83840FFF751BE042C02D14E4926
:1033B4000C20ACE7032CA8D0052CDAD10022494913
:1033C4001820EEE7042C02D148490D209FE7032C76
:1033D400DFD0052CCDD1002243491920E1E7032C8D
:1033E400E5D0052CC5D1002240491A20D9E7042C88
:1033F40002D13F490F207DE7052C03D10022364935
:103404001C20C0E7012C3FF458AF38BD032C9BD0DF
:10341400052CF7D1002236491D20B4E7042C02D133
:103424003449112073E7052CECD100222B491E20CE
:10343400B7E7042C02D13049122068E7032C8AD064
:10344400052CDFD100222B491F20AAE7042C02D12E
:103454002A4913205BE7032CE2D0052CD2D10022A9
:10346400254920209DE7032CE5D0052CCAD1002254
:103474002249212095E7032C02D14FF07C522AE700
:10348400042C02D14FF03F4225E7052C7FF471AFA5
:103494000D4C002221461420FFF754FD0121206821
:1034A40000F002FC0122164B1A7038BD032C29D1FE
:1034B4004FF07C525AE700BFBF000020F091000893
:1034C40000920008BE000020840000209800002024
:1034D40088000020A0000020B4000020A4000020E8
:1034E4009C0000208C00002090000020940000200C
:1034F400B8000020A8000020AC000020B00000208C
:10350400BD000020042C02D14FF03F422EE7052CD1
:103514000AD1A84C0221206800F0F6FB00222146C3
:103524001520FFF75BFDBDE7012C3FF4E1AE38BD8C
:10353400032C02D14FF07C5223E7042C02D14FF02C
:103544003F421EE7052C08D19B4C0321206800F064
:10355400DBFB002221461620E3E7012CE7D1FFE63E
:10356400032C0CD1954C96492068FDF747F918B106
:103574004FF07E52214613E74FF07C52FAE7042CB9
:103584000AD18E4C8E492068FDF738F908B18D4A6E
:10359400F0E74FF03F42EDE7052C0AD1874C0421B8
:1035A400206800F02DFC002221461720FFF74EFD75
:1035B40078E7012CBBD1A8E6032C0CD1824C8049BE
:1035C4002068FDF71BF918B14FF07E522146F7E64B
:1035D4004FF07C52FAE7042C0AD17B4C78492068DE
:1035E400FDF70CF908B1774AF0E74FF03F42EDE7F9
:1035F400052C08D1744D2146286800F001FC0022F6
:1036040029461820D2E7012C91D1C2E6032C0CD113
:103614006E4C6B492068FDF7F1F818B14FF07E52FB
:103624002146DAE64FF07C52FAE7042C0AD1674CC3
:1036340063492068FDF7E2F808B1624AF0E74FF009
:103644003F42EDE7052C08D1604C0621206800F0CC
:10365400D7FB002221461920A8E7012C7FF467AF8D
:10366400A5E6032C0CD15A4C55492068FDF7C6F841
:1036740018B14FF07E522146B7E64FF07C52FAE77C
:10368400042C0AD1524C4E492068FDF7B7F808B112
:103694004C4AF0E74FF03F42EDE7052C08D14C4C83
:1036A4000721206800F0ACFB002221461A207DE7A8
:1036B400012C7FF43CAF87E6032C02D14FF07C52FF
:1036C40032E6042C02D14FF03F422DE6052C7FF464
:1036D40099AE404C002221461B20FFF733FC082101
:1036E400DDE6032C02D14FF07C5288E6042C02D193
:1036F4004FF03F4283E6052C08D1374C092120685E
:1037040000F002FB002221461C200AE7012C7FF472
:103714000EAF19E6032C02D14FF07C527BE6042C49
:1037240002D14FF03F4276E6052C08D12B4C0A21FA
:10373400206800F0E9FA002221461D20F1E6012C60
:103744007FF4F5AE55E6032C0CD1254C1C492068BA
:10375400FDF754F818B14FF07E52214667E64FF05A
:103764007C52FAE7042C0AD11D4C15492068FDF758
:1037740045F808B1134AF0E74FF03F42EDE7052C56
:1037840008D1174C0B21206800F03AFB0022214697
:103794001E200BE7012C7FF4CAAEDCE5032C26D1F6
:1037A400104C07492068FDF729F8E8B14FF07E5224
:1037B400214649E6980000209C0000208800002053
:1037C40000007042000080BF8C00002090000020A8
:1037D40094000020A0000020B4000020B8000020C5
:1037E400A4000020A80000204FF07C52E0E7042C45
:1037F4000AD1384C38492068FDF700F808B1374A37
:10380400D6E74FF03F42D3E7052C08D1314C0C21C9
:10381400206800F0F5FA002221461F20C6E6012C9C
:103824007FF485AEFCE5032C0CD12D4C2A4920688D
:10383400FCF7E4FF18B14FF07E52214611E64FF039
:103844007C52FAE7042C0AD1254C23492068FCF762
:10385400D5FF08B1214AF0E74FF03F42EDE7052CD0
:1038640008D11F4C0D21206800F0CAFA002221461D
:1038740020209BE6012C7FF45AAEDCE5032C0CD10E
:10388400184C15492068FCF7B9FF18B14FF07E5267
:103894002146EEE54FF07C52FAE7042C0AD1114C94
:1038A4000D492068FCF7AAFF08B10C4AF0E74FF075
:1038B4003F42EDE7052C08D10A4C0E21206800F0A8
:1038C4009FFA00222146212070E6012C7FF42FAEBE
:1038D400BEE500BFA800002000007042000080BFC9
:1038E400AC000020B00000202DE9F047A8B1C0438F
:1038F4004FF0834500F03F044FF0824600204FF024
:1039040081474FF080484FF07E594FF07C5A34B9CC
:103914000021FCF713FEBDE8F0870020F8E7E1077B
:1039240005D5514604F0FE04FCF708FEEFE7A207B4
:1039340003D504F0FD044946F6E7630703D504F014
:10394400FB044146F0E7210703D504F0F7043946A8
:10395400EAE7E20603D504F0EF043146E4E7A30600
:1039640003D504F0DF042946DEE70249FCF7E6FD4F
:10397400CEE700BF0000FC412DE9F84F00F03F0402
:103984004FF07C5500204FF07E564FF080474FF0AB
:1039940081484FF082494FF0834ADFF868B03F2CEA
:1039A40003D15946FCF7CAFD0024A10605D55146AA
:1039B40004F01F04FCF7C2FDF1E7E20603D504F0AE
:1039C4002F044946F6E7230703D504F0370441469C
:1039D400F0E7610703D504F03B043946EAE7A207A0
:1039E40003D504F03D043146E4E7E30703D504F0CE
:1039F4003E042946DEE7002CD1D10021FCF79EFDD0
:103A0400BDE8F88F0000FC41C0432DE9F84300F005
:103A14001F044FF0834500204FF082464FF081474A
:103A24004FF080484FF07E5924B90021FCF786FD01
:103A3400BDE8F883E20705D5494604F01E04FCF707
:103A44007DFDF1E7A30703D504F01D044146F6E725
:103A5400610703D504F01B043946F0E7220703D5B8
:103A640004F017043146EAE7E30603D504F00F0433
:103A74002946E4E714F01E0F14BF02490249FCF77B
:103A84005DFDD2E70000F8410000FC412DE9F74F4D
:103A940083463F2400254FF083464FF082474FF082
:103AA40081484FF080494FF07E5A29465846FCF72A
:103AB40091FE0190002853D12B495846FCF78AFE09
:103AC400019A60B931465846FCF7A2FE50B15846F7
:103AD4003146FCF731FD04F01F048346E5E7144644
:103AE400AB46E2E739465846FCF792FE38B15846F1
:103AF4003946FCF721FD04F02F048346D5E74146FF
:103B04005846FCF785FE38B158464146FCF714FD8B
:103B140004F037048346C8E749465846FCF778FE64
:103B240038B158464946FCF707FD04F03B04834688
:103B3400BBE751465846FCF76BFE38B15846514630
:103B4400FCF7FAFC04F03D048346AEE74FF07C51E9
:103B54005846FCF75DFE0028A7D004F03E04BFE7FA
:103B6400204603B0BDE8F08F0000FC412DE9F84F7A
:103B74000546002400264FF083474FF082484FF05B
:103B840081494FF0804A4FF07E5B31462846FCF76E
:103B940021FE002858D12E492846FCF71BFE60B9A7
:103BA40039462846FCF734FE50B128463946FCF71E
:103BB400C3FC44F020040546E7E73F243546E4E728
:103BC40041462846FCF724FE38B128464146FCF716
:103BD400B3FC44F010040546D7E749462846FCF7F1
:103BE40017FE38B128464946FCF7A6FC44F0080401
:103BF4000546CAE751462846FCF70AFE38B128466E
:103C04005146FCF799FC44F004040546BDE75946C7
:103C14002846FCF7FDFD38B128465946FCF78CFCD4
:103C240044F002040546B0E74FF07C512846FCF707
:103C3400EFFD0028A9D028464FF07C51FCF77CFC0E
:103C440044F001040546A0E72046BDE8F88F00BF14
:103C54000000FC4103461F202BB31F2B06D00F2B63
:103C640006D9103BDBB200F00F00F5E700207047E7
:103C7400072B04D9083BDBB200F01700ECE7032B59
:103C840004D9043BDBB200F01B00E5E7012B89BF3C
:103C9400023B03F1FF33DBB200F01D009CBFDBB23B
:103CA40000F01E00D8E770471FB5002302938DF87B
:103CB4000C30BE238DF8043004238DF805108DF8E4
:103CC4000630FFF7E3FE3F238DF8070006210DF1D0
:103CD40005008DF808308DF809308DF80A30EB2492
:103CE40003F032FE074A8DF80B008DF80C4001AB4F
:103CF40003CB1472106051600120FEF783FB04B003
:103D040010BD00BFCD0000201FB500230193029316
:103D14008DF80C30BE238DF8043004238DF8051083
:103D2400334904468DF80630FCF77CFD18B30323B1
:103D34002F4920468DF807308DF808308DF809306A
:103D4400FCF7FAFBFFF7A2FE8DF80A0006210DF13D
:103D5400050003F0F9FDEB24264A8DF80B008DF8DD
:103D64000C4001AB03CB1472106051600120FEF7CC
:103D740049FB04B010BD20492046FCF753FDA0B117
:103D84001D492046FCF7D8FB0446FFF77FFE0323BA
:103D940020468DF807308DF80830FFF777FE3F2373
:103DA4008DF809008DF80A30D0E714492046FCF755
:103DB40039FD70B10323114920468DF80730FCF713
:103DC400BBFBFFF763FE3F238DF808008DF8093035
:103DD400E8E700212046FCF71BFD0028B6D020466A
:103DE400FFF754FE3F238DF807008DF80830EDE708
:103DF4000000B442CD000020000070420000F041F9
:103E04001FB50023019302938DF80C30BE238DF867
:103E1400043004238DF80510274904468DF8063034
:103E2400FCF700FD08B30123234920468DF8073031
:103E34008DF80830FCF780FBFFF798FE8DF8090039
:103E440006210DF1050003F07FFDEB241B4A8DF8DC
:103E54000B008DF80C4001AB03CB14721060516061
:103E64000120FEF7CFFA04B010BD15492046FCF737
:103E7400CFFC70B10123124920468DF80730FCF7BE
:103E84005BFBFCF7D9FCC0B2FFF7E4FE8DF8080039
:103E9400D6E700212046FCF7BBFC0028D0D0204602
:103EA400FCF7CAFCC0B2FFF7D5FE1F238DF807004C
:103EB4008DF80830C4E700BF00007042CD00002038
:103EC4000000F041F8B50646002949D001294AD03E
:103ED40002294BD003294CD0042914BF4FF4806528
:103EE4004FF480450624244F16F0200218BF012207
:103EF4004FF400713846FCF7F9FF01224FF480714A
:103F04001D48FCF7F3FF0120FCF77AFE00224FF472
:103F140080711948FCF7EAFF013C01207600FCF7A8
:103F24006FFE14F0FF04F6B2DED122464FF4807126
:103F34001148FCF7DBFF22464FF400710E48FCF7F2
:103F4400D5FF294601220C48FCF7D0FF0120FCF7DD
:103F540057FE22462946BDE8F8400748FCF7C6BF8D
:103F64004FF48065BEE74FF40065BBE74FF480551E
:103F7400B8E74FF40055B5E7001002402DE9F041D1
:103F84000546884600294ED001294FD002294FD03A
:103F940003294FD004290CBF4FF4007700270624CF
:103FA400254E15F0200218BF01224FF4005130466F
:103FB400FCF79CFF01224FF480513046FCF796FF3A
:103FC4000120FCF71DFE00224FF480513046FCF71F
:103FD4008DFF013C01206D00FCF712FE14F0FF047C
:103FE400EDB2DED122464FF480511348FCF77EFF38
:103FF400114D124B2246B8F1000F18BF1D464FF465
:1040040000512846FCF772FF394601222846FCF786
:104014006DFF0120FCF7F4FD224639462846BDE831
:10402400F041FCF763BF4FF48047B8E74027B6E799
:104034008027B4E72027B2E70018024000040240BA
:1040440070B500224FF4004105462748FCF74EFFA7
:1040540000224FF480412448FCF748FF00224FF42B
:1040640000512148FCF742FF08241F4E2B064CBF89
:10407400012200224FF480413046FCF737FF012231
:104084004FF400511848FCF731FF0120FCF7B8FD4C
:1040940000224FF400511448FCF728FF013C012092
:1040A4006D00FCF7ADFD14F0FF04EDB2DED101228A
:1040B4004FF400410C48FCF719FF0120FCF7A0FD68
:1040C40022464FF400410848FCF710FF22464FF403
:1040D40080410548FCF70AFF2246BDE870404FF4D2
:1040E40000510148FCF702BF0014024070B50022E1
:1040F4004FF4007105462448FCF7F8FE00228021A5
:104104002248FCF7F3FE002240212048FCF7EEFE93
:1041140008241E4E2B064CBF01220022802130466B
:10412400FCF7E4FE012240211848FCF7DFFE0120E1
:10413400FCF766FD002240211448FCF7D7FE013C41
:1041440001206D00FCF75CFD14F0FF04EDB2E1D139
:1041540001224FF400710C48FCF7C8FE0120FCF763
:104164004FFD22464FF400710748FCF7BFFE22467C
:1041740080210648FCF7BAFE2246BDE87040402183
:104184000248FCF7B3BE00BF00180240000C024016
:1041940038B504460D4610F0100218BF0122102154
:1041A4002248FCF7A3FE14F0080218BF0122802164
:1041B4001F48FCF79BFE14F0040218BF01224021A3
:1041C4001B48FCF793FE14F0020218BF01222021C1
:1041D4001748FCF78BFE14F0010218BF01221021CE
:1041E4001348FCF783FE8DB9012220210F48FCF708
:1041F4007DFE0120FCF704FD2A4620210B48FCF734
:1042040075FEBDE838400120FCF7FABC012D0BD146
:104214002A4629460748FCF769FE2846FCF7F0FCC5
:10422400002229460348EAE738BD00BF00080240DF
:10423400000002400004024038B504460D4610F068
:10424400100218BF012202212348FCF74FFE14F08C
:10425400080218BF012201211F48FCF747FE14F091
:10426400040218BF01224FF480511C48FCF73EFEA3
:1042740014F0020218BF01224FF400611748FCF742
:1042840035FE14F0010218BF01224FF48061134877
:10429400FCF72CFE8DB9012204210F48FCF726FE01
:1042A4000120FCF7ADFC2A4604210B48FCF71EFE56
:1042B400BDE838400120FCF7A3BC012D0AD12A46F1
:1042C40008210548FCF712FE2846FCF799FC002259
:1042D4000821EAE738BD00BF000C02400008024094
:1042E4002DE9F047164E044640213046FCF7F8FD10
:1042F400144D814602212846FCF7F2FD8021074631
:104304003046FCF7EDFD042182462846FCF7E8FD23
:104314004FF4807180463046FCF7E2FD08210646E2
:104324002846FCF7DDFD2670E07084F801A084F8CF
:10433400029084F8048067712046BDE8F08700BFCE
:10434400001402400008024007B502AB03E9030071
:104354009DF8023013B19DF8053063BB002204219F
:104364001F48FCF7C3FD012208211D48FCF7BEFDD0
:104374009DF8013013B19DF804301BBB00221021BD
:104384001748FCF7B3FD012220211548FCF7AEFDC8
:104394009DF8003013B19DF80330D3B900220121F8
:1043A4000F48FCF7A3FD012202210D4803B05DF87C
:1043B40004EBFCF79BBD012204210948FCF796FDA0
:1043C4000022D1E7012210210548FCF78FFD0022CD
:1043D400DAE7012202481146FCF788FD0022E3E7F0
:1043E400001002400A460A2301460148FDF7A6BE12
:1043F400380C002084B038B504AC84E80F00149C59
:1044040004ABE21C14A953F8040B8B4242F8040BCE
:10441400F9D1A178601CCD1C0231C9B203F094FA21
:10442400EB226055A378204623441A71A178053104
:10443400C9B2FFF7D7FFBDE8384004B070470000A9
:1044440084B070B59AB01EAC84E80F0064220021D9
:1044540001A89DF8B8502EAE03F0C7FC1EAA01AB0C
:104464001C4610685168083203C4B2422346F7D18F
:104474003F2D00F2E680DFE805F020272A2D3033B7
:1044840036393C3F4245484B4E5154575A5D606360
:1044940066696C6F7275787B7E8184878A8D909350
:1044A40096999C9FA2A5A8ABAEB1B4B7BABDC0C340
:1044B400C6C9CCCFD2D5D8DBDEE19DF878001AB0DE
:1044C400BDE8704004B070479DF87900F7E79DF8A7
:1044D4007A00F4E79DF87B00F1E79DF87C00EEE7B5
:1044E4009DF87D00EBE79DF87E00E8E79DF87F00EE
:1044F400E5E79DF88000E2E79DF88100DFE79DF89D
:104504008200DCE79DF88300D9E79DF88400D6E7B4
:104514009DF88500D3E79DF88600D0E79DF88700D5
:10452400CDE79DF88800CAE79DF88900C7E79DF8A4
:104534008A00C4E79DF88B00C1E79DF88C00BEE7B4
:104544009DF88D00BBE79DF88E00B8E79DF88F00BD
:10455400B5E79DF89000B2E79DF89100AFE79DF8AC
:104564009200ACE79DF89300A9E79DF89400A6E7B4
:104574009DF89500A3E79DF89600A0E79DF89700A5
:104584009DE79DF898009AE79DF8990097E79DF8B4
:104594009A0094E79DF89B0091E79DF89C008EE7B4
:1045A4009DF89D008BE79DF89E0088E79DF89F008D
:1045B40085E79DF8A00082E79DF8A1007FE79DF8BC
:1045C400A2007CE79DF8A30079E79DF8A40076E7B4
:1045D4009DF8A50073E79DF8A60070E79DF8A70075
:1045E4006DE79DF8A8006AE79DF8A90067E79DF8C4
:1045F400AA0064E79DF8AB0061E79DF8AC005EE7B4
:104604009DF8AD005BE79DF8AE0058E79DF8AF005C
:1046140055E79DF8B00052E79DF8B1004FE79DF8CB
:10462400B2004CE79DF8B30049E79DF8B40046E7B3
:104634009DF8B50043E79DF8B60040E79DF8B70044
:104644003DE7024803F04EFC002038E714930008CD
:1046540084B008B50DF1080E8EE80F009DF84830BF
:104664003F2B00F2E580DFE803F0E0DDDAD7D4D1B8
:10467400CECBC8C5C2BFBCB9B6B3B0ADAAA7A4A1BE
:104684009E9B9895928F8C898683807D7A777471AE
:104694006E6B6865625F5C595653504D4A4744419E
:1046A4003E3B3835322F2C2926209DF80800BDE8E2
:1046B400084004B070479DF80900F8E79DF80A0027
:1046C400F5E79DF80B00F2E79DF80C00EFE79DF885
:1046D4000D00ECE79DF80E00E9E79DF80F00E6E712
:1046E4009DF81000E3E79DF81100E0E79DF8120043
:1046F400DDE79DF81300DAE79DF81400D7E79DF88D
:104704001500D4E79DF81600D1E79DF81700CEE711
:104714009DF81800CBE79DF81900C8E79DF81A002A
:10472400C5E79DF81B00C2E79DF81C00BFE79DF894
:104734001D00BCE79DF81E00B9E79DF81F00B6E711
:104744009DF82000B3E79DF82100B0E79DF8220012
:10475400ADE79DF82300AAE79DF82400A7E79DF89C
:104764002500A4E79DF82600A1E79DF827009EE711
:104774009DF828009BE79DF8290098E79DF82A00FA
:1047840095E79DF82B0092E79DF82C008FE79DF8A4
:104794002D008CE79DF82E0089E79DF82F0086E711
:1047A4009DF8300083E79DF8310080E79DF83200E2
:1047B4007DE79DF833007AE79DF8340077E79DF8AC
:1047C400350074E79DF8360071E79DF837006EE711
:1047D4009DF838006BE79DF8390068E79DF83A00CA
:1047E40065E79DF83B0062E79DF83C005FE79DF8B4
:1047F4003D005CE79DF83E0059E79DF83F0056E711
:104804009DF8400053E79DF8410050E79DF84200B1
:104814004DE79DF843004AE79DF8440047E79DF8BB
:10482400450044E79DF8460041E79DF847003EE710
:10483400024803F057FB002039E700BF1493000837
:1048440084B008B50DF1080E8EE80F009DF84830CD
:104854001F2B74D8DFE803F01016191C1F2225281B
:104864002B2E3134373A3D404346494C4F5255582C
:104874005B5E6164676A6D709DF80900BDE808407D
:1048840004B070479DF80B00F8E79DF80D00F5E7BC
:104894009DF80F00F2E79DF81100EFE79DF8130073
:1048A400ECE79DF81500E9E79DF81700E6E79DF8A9
:1048B4001900E3E79DF81B00E0E79DF81D00DDE724
:1048C4009DF81F00DAE79DF82100D7E79DF8230043
:1048D400D4E79DF82500D1E79DF82700CEE79DF8A1
:1048E4002900CBE79DF82B00C8E79DF82D00C5E70C
:1048F4009DF82F00C2E79DF83100BFE79DF8330013
:10490400BCE79DF83500B9E79DF83700B6E79DF898
:104914003900B3E79DF83B00B0E79DF83D00ADE7F3
:104924009DF83F00AAE79DF84100A7E79DF84300E2
:10493400A4E79DF84500A1E79DF847009EE70248DB
:1049440003F0D0FA002099E71493000810B5204C26
:1049540000212078FFF7B6FA60780121FFF7B2FA58
:10496400A0780221FFF7AEFAE0780321FFF7AAFA54
:1049740020790421FFF7A6FA60790021FFF708FCEB
:104984000121A079FFF704FCE079FFF759FB207AB5
:104994000021FFF7F3FA607A0121FFF7EFFAA07A1A
:1049A4000221FFF7EBFAE07A0321FFF7E7FA207B15
:1049B4000421FFF7E3FA607B0021FFF73DFCA07BB5
:1049C4000121FFF739FCE07BBDE81040FFF78EBB07
:1049D400500B0020F0B543788FB004466C2B00F2E6
:1049E400C482DFE813F06D009200A800C000D80074
:1049F400F0000801200138014901610179019101A8
:104A0400A901C101C202D901DD01E101E501E90108
:104A1400EE01F301F801FD0102020702C202C20223
:104A2400C2020C02110216021B02200227022C02EF
:104A3400310236023B02400245024A024F0254024E
:104A440059025E02630268026D02720277027C02FE
:104A5400810286028B02900295029A029F02A402AE
:104A6400C202C202C202A902C402DA02F0020603AE
:104A74001C03320348035E0374038A03C202C202A6
:104A8400C202A003B603CC03E203F8030E04240419
:104A94005F0475048B04A104B704CD04E304F90492
:104AA4000F0525053B05510567057D059305A905FA
:104AB400BF05D5050F0625063B06510667067D068C
:104AC400BE23037000234370D94BC21C03F1280199
:104AD40053F8040B8B4242F8040BF9D11B88601C79
:104AE4001380A178CD1C0231C9B202F02DFFEB2254
:104AF40060552046A37823441A71A1780531C9B2C0
:104B04000FB0BDE8F040FFF76DBC14F8030F0021AF
:104B1400FFF7D8F90123224640F6B821A02002F07D
:104B2400F7F9042322464FF42861A0200FB0BDE812
:104B3400F04002F0EDB90025861C0135EDB229469E
:104B440016F8010FFFF7BEF9042DF6D103342B46F6
:104B5400224640F6B921A02002F0DAF92B4622467B
:104B640040F68421E1E70025861C0135EDB2294693
:104B740016F8010FFFF7A6F9042DF6D103342B46DE
:104B8400224640F6B921A02002F0C2F92B46224663
:104B940040F68821C9E70021C078FFF7F9FA2079A7
:104BA4000121FFF7F5FA0334A078FFF749FA03234C
:104BB400224640F6BD21A02002F0AAF90423224691
:104BC40040F68C21B1E70021C078FFF7E1FA2079A3
:104BD4000121FFF7DDFA0334A078FFF731FA03234C
:104BE400224640F6BD21A02002F092F90423224679
:104BF4004FF4296199E70021C078FFF7C9FA2079B9
:104C04000121FFF7C5FA0334A078FFF719FA03234B
:104C1400224640F6BD21A02002F07AF90423224660
:104C240040F6942181E70021C078FFF7B1FA20799A
:104C34000121FFF7ADFA0334A078FFF701FA03234B
:104C4400224640F6BD21A02002F062F90423224648
:104C540040F6982169E714F8030F0021FFF78EF955
:104C6400012322464FF42C61A02002F051F90423C1
:104C7400224640F69C2158E70025861C0135EDB2FA
:104C8400294616F8010FFFF779F9042DF6D10334FC
:104C94002B46224640F6C121A02002F039F92B46CA
:104CA40022464FF42A6140E70025861C0135EDB207
:104CB400294616F8010FFFF761F9042DF6D10334E4
:104CC4002B46224640F6C121A02002F021F92B46B2
:104CD400224640F6A42128E70021C078FFF7ACFA69
:104CE40020790121FFF7A8FA0334A078FFF7FEF931
:104CF4000323224640F6C521A02002F009F904232B
:104D0400224640F6A82110E70021C078FFF794FA64
:104D140020790121FFF790FA0334A078FFF7E6F930
:104D24000323224640F6C521A02002F0F1F8042313
:104D3400224640F6AC21F8E60021C078FFF77CFA61
:104D440020790121FFF778FA0334A078FFF7CEF930
:104D54000323224640F6C521A02002F0D9F80423FB
:104D640022464FF42B61E0E60021C078FFF764FA95
:104D740020790121FFF760FA0334A078FFF7B6F930
:104D84000323224640F6C521A02002F0C1F80423E3
:104D9400224640F6B421C8E64023C21C0021C4E6E2
:104DA4004023C21C1946C0E64023C21C8021BCE635
:104DB4004023C21CC021B8E64023C21C4FF48071BA
:104DC400B3E64023C21C4FF4A071AEE64023C21CDC
:104DD4004FF4C071A9E64023C21C4FF4E071A4E66D
:104DE4004023C21C4FF400719FE64023C21C4FF4C1
:104DF40010719AE64023C21C4FF4207195E64023BB
:104E0400C21C4FF4307190E64023C21C4FF4407131
:104E14008BE64023C21C4FF4507186E64023C21C2B
:104E24004FF4607181E64023C21C4FF470717CE63C
:104E3400A60700204023C21C4FF4806175E640237E
:104E4400C21C4FF4886170E64023C21C4FF4906189
:104E54006BE64023C21C4FF4986166E64023C21CF3
:104E64004FF4A06161E64023C21C4FF4A8615CE6E4
:104E74004023C21C4FF4B06157E64023C21C4FF4D8
:104E8400B86152E64023C21C4FF4C0614DE6402392
:104E9400C21C4FF4C86148E64023C21C4FF4D061E1
:104EA40043E64023C21C4FF4D8613EE64023C21CB3
:104EB4004FF4E06139E64023C21C4FF4E86134E664
:104EC4004023C21C4FF4F0612FE64023C21C4FF470
:104ED400F8612AE64023C21C4FF4006125E6402312
:104EE400C21C4FF4046120E64023C21C4FF4086145
:104EF4001BE64023C21C4FF40C6116E64023C21C7F
:104F04004FF4106111E64023C21C4FF414610CE607
:104F14004023C21C4FF4186107E64023C21C4FF41F
:104F24001C6102E64023C21C4FF42061FDE54023CE
:104F3400C21C4FF42461F8E56F46C8490C90D1F8BF
:104F440000C0D1F804E08A68CB6801F1100501F1D2
:104F540040043E4628686968083503C6A5423746BA
:104F6400F7D160467146FFF745FA0FB0F0BD6F46C2
:104F7400BB490C90D1F800C0D1F804E08A68CB6832
:104F840001F1100501F140043E46286869680835BE
:104F940003C6A5423746F7D1E3E76F46B1490C9003
:104FA400D1F800C0D1F804E08A68CB6801F110059B
:104FB40001F140043E4628686968083503C6A542E5
:104FC4003746F7D1CDE76F46A7490C90D1F800C01A
:104FD400D1F804E08A68CB6801F1100501F14004BE
:104FE4003E4628686968083503C6A5423746F7D1A6
:104FF400B7E76F469D490C90D1F800C0D1F804E0A2
:105004008A68CB6801F1100501F140043E46286826
:105014006968083503C6A5423746F7D1A1E76F464C
:1050240093490C90D1F800C0D1F804E08A68CB68A9
:1050340001F1100501F140043E462868696808350D
:1050440003C6A5423746F7D18BE76F4689490C90D2
:10505400D1F800C0D1F804E08A68CB6801F11005EA
:1050640001F140043E4628686968083503C6A54234
:105074003746F7D175E76F467F490C90D1F800C0E9
:10508400D1F804E08A68CB6801F1100501F140040D
:105094003E4628686968083503C6A5423746F7D1F5
:1050A4005FE76F4675490C90D1F800C0D1F804E071
:1050B4008A68CB6801F1100501F140043E46286876
:1050C4006968083503C6A5423746F7D149E76F46F4
:1050D4006B490C90D1F800C0D1F804E08A68CB6821
:1050E40001F1100501F140043E462868696808355D
:1050F40003C6A5423746F7D133E76F4661490C90A2
:10510400D1F800C0D1F804E08A68CB6801F1100539
:1051140001F140043E4628686968083503C6A54283
:105124003746F7D11DE76F4657490C90D1F800C0B8
:10513400D1F804E08A68CB6801F1100501F140045C
:105144003E4628686968083503C6A5423746F7D144
:1051540007E76F464D490C90D1F800C0D1F804E040
:105164008A68CB6801F1100501F140043E462868C5
:105174006968083503C6A5423746F7D1F1E66F469C
:1051840043490C90D1F800C0D1F804E08A68CB6898
:1051940001F1100501F140043E46286869680835AC
:1051A40003C6A5423746F7D1DBE66F4639490C9072
:1051B400D1F800C0D1F804E08A68CB6801F1100589
:1051C40001F140043E4628686968083503C6A542D3
:1051D4003746F7D1C5E66F462F490C90D1F800C089
:1051E400D1F804E08A68CB6801F1100501F14004AC
:1051F4003E4628686968083503C6A5423746F7D194
:10520400AFE66F4625490C90D1F800C0D1F804E010
:105214008A68CB6801F1100501F140043E46286814
:105224006968083503C6A5423746F7D199E66F4643
:105234001B490C90D1F800C0D1F804E08A68CB680F
:1052440001F1100501F140043E46286869680835FB
:1052540003C6A5423746F7D183E600BFD007002036
:10526400E0020020100B0020A0030020E001002039
:10527400100A0020A00B0020E00600206007002098
:1052840020060020D00A002020070020100900205A
:1052940060040020A0050020600B0020E004002032
:1052A400600100206F46C5490C90D1F800C0D1F8C8
:1052B40004E08A68CB6801F1100501F140043E4620
:1052C40028686968083503C6A5423746F7D148E619
:1052D4006F46BB490C90D1F800C0D1F804E08A684D
:1052E400CB6801F1100501F140043E462868696865
:1052F400083503C6A5423746F7D132E66F46B149B1
:105304000C90D1F800C0D1F804E08A68CB6801F1B0
:10531400100501F140043E4628686968083503C653
:10532400A5423746F7D11CE66F46A7490C90D1F841
:1053340000C0D1F804E08A68CB6801F1100501F1DE
:1053440040043E4628686968083503C6A5423746C6
:10535400F7D106E66F469D490C90D1F800C0D1F80C
:1053640004E08A68CB6801F1100501F140043E466F
:1053740028686968083503C6A5423746F7D1F0E5C1
:105384006F4693490C90D1F800C0D1F804E08A68C4
:10539400CB6801F1100501F140043E4628686968B4
:1053A400083503C6A5423746F7D1DAE56F46894981
:1053B4000C90D1F800C0D1F804E08A68CB6801F100
:1053C400100501F140043E4628686968083503C6A3
:1053D400A5423746F7D1C4E56F467F490C90D1F812
:1053E40000C0D1F804E08A68CB6801F1100501F12E
:1053F40040043E4628686968083503C6A542374616
:10540400F7D1AEE56F4675490C90D1F800C0D1F8DC
:1054140004E08A68CB6801F1100501F140043E46BE
:1054240028686968083503C6A5423746F7D198E568
:105434006F466B490C90D1F800C0D1F804E08A683B
:10544400CB6801F1100501F140043E462868696803
:10545400083503C6A5423746F7D182E56F46614950
:105464000C90D1F800C0D1F804E08A68CB6801F14F
:10547400100501F140043E4628686968083503C6F2
:10548400A5423746F7D16CE56F4657490C90D1F8E1
:1054940000C0D1F804E08A68CB6801F1100501F17D
:1054A40040043E4628686968083503C6A542374665
:1054B400F7D156E56F464D490C90D1F800C0D1F8AC
:1054C40004E08A68CB6801F1100501F140043E460E
:1054D40028686968083503C6A5423746F7D140E510
:1054E4006F4643490C90D1F800C0D1F804E08A68B3
:1054F400CB6801F1100501F140043E462868696853
:10550400083503C6A5423746F7D12AE56F4639491F
:105514000C90D1F800C0D1F804E08A68CB6801F19E
:10552400100501F140043E4628686968083503C641
:10553400A5423746F7D114E56F462F490C90D1F8B0
:1055440000C0D1F804E08A68CB6801F1100501F1CC
:1055540040043E4628686968083503C6A5423746B4
:10556400F7D1FEE46F4625490C90D1F800C0D1F87C
:1055740004E08A68CB6801F1100501F140043E465D
:1055840028686968083503C6A5423746F7D1E8E4B8
:105594006F461B490C90D1F800C0D1F804E08A682A
:1055A400CB6801F1100501F140043E4628686968A2
:1055B400083503C6A5423746F7D1D2E49008002047
:1055C400500800202002002090090020A0040020A0
:1055D400E00300201008002020010020500A0020D1
:1055E400E00500206002002060030020A0010020EC
:1055F40020030020D00900202004002060050020A2
:10560400A00200206F4641490C90D1F800C0D1F8A7
:1056140004E08A68CB6801F1100501F140043E46BC
:1056240028686968083503C6A5423746F7D198E467
:105634006F4637490C90D1F800C0D1F804E08A686D
:10564400CB6801F1100501F140043E462868696801
:10565400083503C6A5423746F7D182E46F462D4983
:105664000C90D1F800C0D1F804E08A68CB6801F14D
:10567400100501F140043E4628686968083503C6F0
:10568400A5423746F7D16CE46F4623490C90D1F814
:1056940000C0D1F804E08A68CB6801F1100501F17B
:1056A40040043E4628686968083503C6A542374663
:1056B400F7D156E46F4619490C90D1F800C0D1F8DF
:1056C40004E08A68CB6801F1100501F140043E460C
:1056D40028686968083503C6A5423746F7D140E40F
:1056E4006F460F490C90D1F800C0D1F804E08A68E5
:1056F400CB6801F1100501F140043E462868696851
:10570400083503C6A5423746F7D12AE460060020CF
:10571400A00600202005002050090020900A002047
:10572400D00800202DE9F0410446A8B04578642251
:1057340000210FA802F059FB237828AA8DF83C30E9
:10574400A3788DF83D508DF83E301A4423441B79DC
:1057540002F8603C6C2D01F2A383DFE815F06D00C4
:1057640079009B0009017201E9013C028F02E20207
:10577400FB028703EF03420495040B05A10B5E05AE
:1057840074058A05A005B605CC05E205F8050E06E4
:1057940024063A06A10BA10BA10B500666067C0653
:1057A4009206CF06E506FB06110727073D075307B8
:1057B40069077F079507AB07C107D707ED070308FC
:1057C40019082F0845085B089708AD08C308D908CD
:1057D400EF0805091B093109A10BA10BA10B47090E
:1057E400540961096E097B0988099509A209AF0961
:1057F400BC09C909A10BA10BA10BD609E309F00946
:10580400FD090A0A170A240A310A3E0A830A900A81
:105814009D0AAA0AB70AC40AD10ADE0AEB0AF80AE0
:10582400050B120B1F0B2C0B390B460B530B600B88
:105834006D0B7A0B870B940BE278AE490DF13F00A8
:1058440002F0C8FA0FA8FFF7C5F828B0BDE8F08148
:10585400EE46E278A84BA94D9A71E37805F110065B
:105864000C93D5F80080D5F804C0AA68EB684035DD
:10587400774630687168083603C7AE42BE46F7D132
:1058840040466146FEF7DCFDE070A2782146053211
:105894000FA8D5E7EE46D4F80320974B984DC3F8EC
:1058A4000720E37805F110060C93D5F80080D5F8AD
:1058B40004C0AA68EB6840357746306871680836DA
:1058C40003C7AE42BE46F7D140466146FEF7B8FD77
:1058D400EE4623798B4DE0700C93D5F80080D5F813
:1058E40004C0AA68EB6805F11006403577463068B5
:1058F4007168083603C7AE42BE46F7D140466146DA
:10590400FEF79EFDEE4663797F4D20710C93D5F82A
:105914000080D5F804C0AA68EB6805F1100640358C
:10592400774630687168083603C7AE42BE46F7D181
:1059340040466146FEF784FDEE46A379734D6071DF
:105944000C93D5F80080D5F804C0AA68EB6805F17B
:1059540010064035774630687168083603C7AE4292
:10596400BE46F7D140466146FEF76AFDA0718CE75A
:10597400EE46D4F80320604B654DC3F80B20E37862
:1059840005F110060C93D5F80080D5F804C0AA6878
:10599400EB684035774630687168083603C7AE4215
:1059A400BE46F7D140466146FEF74AFDEE462379EE
:1059B400584DE0700C93D5F80080D5F804C0AA685F
:1059C400EB6805F110064035774630687168083693
:1059D40003C7AE42BE46F7D140466146FEF730FDEE
:1059E400EE4663794C4D20710C93D5F80080D5F8C0
:1059F40004C0AA68EB6805F11006403577463068A4
:105A04007168083603C7AE42BE46F7D140466146C8
:105A1400FEF716FDEE46A379404D60710C93D5F860
:105A24000080D5F804C0AA68EB6805F1100640357B
:105A3400774630687168083603C7AE42BE46F7D170
:105A440090E72346EE4633F8031F354A354D11805F
:105A54009B7805F110069370E37840350C9355F864
:105A6400408C55F83CCC55F8382C55F8343C7746E6
:105A740030687168083603C7AE42BE46F7D1404667
:105A84006146FEF7DDFEEE462379274DE0700C9368
:105A9400D5F80080D5F804C0AA68EB6805F11006B3
:105AA4004035774630687168083603C7AE42BE4653
:105AB400F7D140466146FEF7C3FEEE4663791B4DBF
:105AC40020710C93D5F80080D5F804C0AA68EB685F
:105AD40005F110064035774630687168083603C70B
:105AE400AE42BE46F7D140466146FEF7B1FD607155
:105AF400CBE600BFA6070020A0070020D0070020A7
:105B0400E0020020100B0020A0030020E001002090
:105B1400100A0020A00B0020E006002060070020EF
:105B2400AF07002020060020D00A00202007002014
:105B34002346EE4633F8031FBA4ABB4D11809B78C7
:105B440005F110069370E37840350C9355F8408CBA
:105B540055F83CCC55F8382C55F8343C7746306829
:105B64007168083603C7AE42BE46F7D14046614667
:105B7400FEF766FEEE462379AC4DE0700C93D5F843
:105B84000080D5F804C0AA68EB6805F1100640351A
:105B9400774630687168083603C7AE42BE46F7D10F
:105BA40040466146FEF74CFEEE466379A04D2071F7
:105BB4000C93D5F80080D5F804C0AA68EB6805F109
:105BC40010064035774630687168083603C7AE4220
:105BD400BE46F7D187E72346EE4633F8031F954ABE
:105BE400954D11809B7805F110069370E37840354C
:105BF4000C9355F8408C55F83CCC55F8382C55F896
:105C0400343C774630687168083603C7AE42BE46F6
:105C1400F7D140466146FEF713FEEE462379874DE1
:105C2400E0700C93D5F80080D5F804C0AA68EB683E
:105C340005F110064035774630687168083603C7A9
:105C4400AE42BE46F7D140466146FEF7F9FDEE4648
:105C540063797B4D20710C93D5F80080D5F804C08E
:105C6400AA68EB6805F1100640357746306871681C
:105C7400083603C7AE42BE46F7D134E72346EE46A4
:105C840033F8031F6F4A704D11809B7805F110069D
:105C94009370E37840350C9355F8408C55F83CCC20
:105CA40055F8382C55F8343C774630687168083616
:105CB40003C7AE42BE46F7D140466146FEF7C0FD7B
:105CC400EE462379614DE0700C93D5F80080D5F849
:105CD40004C0AA68EB6805F11006403577463068C1
:105CE4007168083603C7AE42BE46F7D140466146E6
:105CF400FEF7A6FDEE466379554D20710C93D5F859
:105D04000080D5F804C0AA68EB6805F11006403598
:105D1400774630687168083603C7AE42BE46F7D18D
:105D2400E1E6EE46E2784B4B4B4DDA76E37805F14B
:105D340010060C93D5F80080D5F804C0AA68EB6867
:105D44004035774630687168083603C7AE42BE46B0
:105D5400F7D195E5EE46D4F803203E4B3F4DDA618A
:105D6400E37805F110060C93D5F80080D5F804C04B
:105D7400AA68EB684035774630687168083603C70F
:105D8400AE42BE46F7D140466146FEF759FBEE46A9
:105D94002379334DE0700C93D5F80080D5F804C016
:105DA400AA68EB6805F110064035774630687168DB
:105DB400083603C7AE42BE46F7D140466146FEF7F9
:105DC4003FFBEE466379274D20710C93D5F8008094
:105DD400D5F804C0AA68EB6805F11006403577468B
:105DE40030687168083603C7AE42BE46F7D14046F4
:105DF4006146FEF725FBEE46A3791B4D60710C93BB
:105E0400D5F80080D5F804C0AA68EB6805F110063F
:105E14004035774630687168083603C7AE42BE46DF
:105E2400F7D19FE5B207002010090020600400208C
:105E3400A0050020B5070020600B0020E00400202E
:105E440060010020B80700209008002050080020BE
:105E540020020020A007002090090020A0040020B8
:105E6400E00300201008002020010020EE46D4F8B2
:105E74000320AF4BAF4D1A62E37805F110060C9383
:105E8400D5F80080D5F804C0AA68EB684035774699
:105E940030687168083603C7AE42BE46F7D1404643
:105EA4006146FEF7CDFAEE462379A34DE0700C93DC
:105EB400D5F80080D5F804C0AA68EB6805F110068F
:105EC4004035774630687168083603C7AE42BE462F
:105ED400F7D140466146FEF7B3FAEE466379974D33
:105EE40020710C93D5F80080D5F804C0AA68EB683B
:105EF40005F110064035774630687168083603C7E7
:105F0400AE42BE46F7D140466146FEF799FAEE46E8
:105F1400A3798B4D60710C93D5F80080D5F804C03B
:105F2400AA68EB6805F11006403577463068716859
:105F3400083603C7AE42BE46F7D113E52346EE4604
:105F440033F8031F7F4A804D11809B7805F11006BA
:105F54009370E37840350C9355F8408C55F83CCC5D
:105F640055F8382C55F8343C774630687168083653
:105F740003C7AE42BE46F7D140466146FEF760FC19
:105F8400EE462379714DE0700C93D5F80080D5F876
:105F940004C0AA68EB6805F11006403577463068FE
:105FA4007168083603C7AE42BE46F7D14046614623
:105FB400FEF746FCEE466379654D20710C93D5F8E7
:105FC4000080D5F804C0AA68EB6805F110064035D6
:105FD400774630687168083603C7AE42BE46F7D1CB
:105FE40081E52346EE4633F8031F5A4A5A4D118081
:105FF4009B7805F110069370E37840350C9355F8BF
:10600400408C55F83CCC55F8382C55F8343C774640
:1060140030687168083603C7AE42BE46F7D14046C1
:106024006146FEF70DFCEE4623794C4DE0700C936F
:10603400D5F80080D5F804C0AA68EB6805F110060D
:106044004035774630687168083603C7AE42BE46AD
:10605400F7D140466146FEF7F3FBEE466379404DC7
:1060640020710C93D5F80080D5F804C0AA68EB68B9
:1060740005F110064035774630687168083603C765
:10608400AE42BE46F7D12EE52346EE4633F8031F53
:10609400344A354D11809B7805F110069370E378EE
:1060A40040350C9355F8408C55F83CCC55F8382CB9
:1060B40055F8343C774630687168083603C7AE42F9
:1060C400BE46F7D140466146FEF7BAFBEE46237959
:1060D400264DE0700C93D5F80080D5F804C0AA686A
:1060E400EB6805F11006403577463068716808366C
:1060F40003C7AE42BE46F7D140466146FEF7A0FB59
:10610400EE4663791A4D20710C93D5F80080D5F8CA
:1061140004C0AA68EB6805F110064035774630687C
:106124007168083603C7AE42BE46F7D1DBE400BF50
:10613400A0070020500A0020E00500206002002093
:1061440060030020C4070020A001002020030020D9
:10615400D0090020C707002020040020600500208B
:10616400A0020020CA07002060060020A00600202C
:10617400200500202346EE4633F8031FCC4ACD4DBC
:1061840011809B7805F110069370E37840350C93E9
:1061940055F8408C55F83CCC55F8382C55F8343C1F
:1061A400774630687168083603C7AE42BE46F7D1F9
:1061B40040466146FEF744FBEE462379BE4DE0704F
:1061C4000C93D5F80080D5F804C0AA68EB6805F1F3
:1061D40010064035774630687168083603C7AE420A
:1061E400BE46F7D140466146FEF72AFBEE46637988
:1061F400B24D20710C93D5F80080D5F804C0AA687C
:10620400EB6805F11006403577463068716808364A
:1062140003C7AE42BE46F7D165E4A94AE31C433442
:1062240053F8041BA34242F8041BF9D1A44B0DF10B
:106234003F0203F1400153F8040B8B4242F8040B74
:10624400F9D1FFF7FFBA9F4AE31C433453F8041B08
:10625400A34242F8041BF9D19A4B0DF13F0203F11A
:10626400400153F8040B8B4242F8040BF9D1FFF7B9
:10627400E9BA954AE31C433453F8041BA34242F899
:10628400041BF9D1904B0DF13F0203F1400153F887
:10629400040B8B4242F8040BF9D1FFF7D3BA8B4AB3
:1062A400E31C433453F8041BA34242F8041BF9D102
:1062B400864B0DF13F0203F1400153F8040B8B426E
:1062C40042F8040BF9D1FFF7BDBA814AE31C433409
:1062D40053F8041BA34242F8041BF9D17C4B0DF183
:1062E4003F0203F1400153F8040B8B4242F8040BC4
:1062F400F9D1FFF7A7BA774AE31C433453F8041BD8
:10630400A34242F8041BF9D1724B0DF13F0203F191
:10631400400153F8040B8B4242F8040BF9D1FFF708
:1063240091BA6D4AE31C433453F8041BA34242F868
:10633400041BF9D1684B0DF13F0203F1400153F8FE
:10634400040B8B4242F8040BF9D1FFF77BBA634A82
:10635400E31C433453F8041BA34242F8041BF9D151
:106364005E4B0DF13F0203F1400153F8040B8B42E5
:1063740042F8040BF9D1FFF765BA594AE31C4334D8
:1063840053F8041BA34242F8041BF9D1544B0DF1FA
:106394003F0203F1400153F8040B8B4242F8040B13
:1063A400F9D1FFF74FBA4F4AE31C433453F8041BA7
:1063B400A34242F8041BF9D14A4B0DF13F0203F109
:1063C400400153F8040B8B4242F8040BF9D1FFF758
:1063D40039BA454AE31C433453F8041BA34242F838
:1063E400041BF9D1404B0DF13F0203F1400153F876
:1063F400040B8B4242F8040BF9D1FFF723BA3B4A52
:10640400E31C433453F8041BA34242F8041BF9D1A0
:10641400364B0DF13F0203F1400153F8040B8B425C
:1064240042F8040BF9D1FFF70DBA314AE31C4334A7
:1064340053F8041BA34242F8041BF9D12C4B0DF171
:106444003F0203F1400153F8040B8B4242F8040B62
:10645400F9D1FFF7F7B9274AE31C433453F8041B77
:10646400A34242F8041BF9D1224B0DF13F0203F180
:10647400400153F8040B8B4242F8040BF9D1FFF7A7
:10648400E1B91D4AE31C433453F8041BA34242F808
:10649400041BF9D1184B0DF13F0203F1400153F8ED
:1064A400040B8B4242F8040BF9D1FFF7CBB900BFC0
:1064B400CD07002050090020900A0020D0080020B9
:1064C400D0070020E0020020100B0020A0030020D1
:1064D400E0010020100A0020A00B0020E0060020AC
:1064E4006007002020060020D00A0020200700209A
:1064F4001009002060040020A0050020D04AE31CFD
:10650400433453F8041BA34242F8041BF9D1CC4B87
:106514000DF13F0203F1400153F8040B8B4242F8A2
:10652400040BF9D1FFF78EB9C64AE31C433453F880
:10653400041BA34242F8041BF9D1C24B0DF13F02E4
:1065440003F1400153F8040B8B4242F8040BF9D1D8
:10655400FFF778B9BC4AE31C433453F8041BA34245
:1065640042F8041BF9D1B84B0DF13F0203F140018D
:1065740053F8040B8B4242F8040BF9D1FFF762B9CC
:10658400B24AE31C433453F8041BA34242F8041BED
:10659400F9D1AE4B0DF13F0203F1400153F8040B66
:1065A4008B4242F8040BF9D1FFF74CB9A84AE31C1B
:1065B400433453F8041BA34242F8041BF9D1A44BFF
:1065C4000DF13F0203F1400153F8040B8B4242F8F2
:1065D400040BF9D1FFF736B99E4AE31C433453F850
:1065E400041BA34242F8041BF9D19A4B0DF13F025C
:1065F40003F1400153F8040B8B4242F8040BF9D128
:10660400FFF720B9944AE31C433453F8041BA34214
:1066140042F8041BF9D1904B0DF13F0203F1400104
:1066240053F8040B8B4242F8040BF9D1FFF70AB973
:106634008A4AE31C433453F8041BA34242F8041B64
:10664400F9D1864B0DF13F0203F1400153F8040BDD
:106654008B4242F8040BF9D1FFF7F4B8804AE31CEB
:10666400433453F8041BA34242F8041BF9D17C4B76
:106674000DF13F0203F1400153F8040B8B4242F841
:10668400040BF9D1FFF7DEB8764AE31C433453F820
:10669400041BA34242F8041BF9D1724B0DF13F02D3
:1066A40003F1400153F8040B8B4242F8040BF9D177
:1066B400FFF7C8B86C4AE31C433453F8041BA342E5
:1066C40042F8041BF9D1684B0DF13F0203F140017C
:1066D40053F8040B8B4242F8040BF9D1FFF7B2B81C
:1066E400624AE31C433453F8041BA34242F8041BDC
:1066F400F9D15E4B0DF13F0203F1400153F8040B55
:106704008B4242F8040BF9D1FFF79CB8584AE31CBA
:10671400433453F8041BA34242F8041BF9D1544BED
:106724000DF13F0203F1400153F8040B8B4242F890
:10673400040BF9D1FFF786B84E4AE31C433453F8EF
:10674400041BA34242F8041BF9D14A4B0DF13F024A
:1067540003F1400153F8040B8B4242F8040BF9D1C6
:10676400FFF770B8444AE31C433453F8041BA342B4
:1067740042F8041BF9D1404B0DF13F0203F14001F3
:1067840053F8040B8B4242F8040BF9D1FFF75AB8C3
:106794003A4AE31C433453F8041BA34242F8041B53
:1067A400F9D1364B0DF13F0203F1400153F8040BCC
:1067B4008B4242F8040BF9D1FFF744B8304AE31C8A
:1067C400433453F8041BA34242F8041BF9D12C4B65
:1067D4000DF13F0203F1400153F8040B8B4242F8E0
:1067E400040BF9D1FFF72EB8264AE31C433453F8BF
:1067F400041BA34242F8041BF9D1224B0DF13F02C2
:1068040003F1400153F8040B8B4242F8040BF9D115
:10681400FFF718B81C4AE31C433453F8041BA34283
:1068240042F8041BF9D1184B0DF13F0203F140016A
:1068340053F8040B8B4242F8040BF9D1FFF702B86A
:10684400600B0020E004002060010020900800207C
:10685400500800202002002090090020A0040020FD
:10686400E00300201008002020010020500A00202E
:10687400E00500206002002060030020A001002049
:1068840020030020D009002020040020D94AE31C62
:10689400433453F8041BA34242F8041BF9D1D54BEB
:1068A4000DF13F0203F1400153F8040B8B4242F80F
:1068B400040BF9D1FEF7C6BFCF4AE31C433453F8A7
:1068C400041BA34242F8041BF9D1CB4B0DF13F0248
:1068D40003F1400153F8040B8B4242F8040BF9D145
:1068E400FEF7B0BFC54AE31C433453F8041BA3426C
:1068F40042F8041BF9D1C14B0DF13F0203F14001F1
:1069040053F8040B8B4242F8040BF9D1FEF79ABFFB
:10691400BB4AE31C433453F8041BA34242F8041B50
:10692400F9D1B74B0DF13F0203F1400153F8040BC9
:106934008B4242F8040BF9D1FEF784BFB14AE31C41
:10694400433453F8041BA34242F8041BF9D1AD4B62
:106954000DF13F0203F1400153F8040B8B4242F85E
:10696400040BF9D1FEF76EBFA74AE31C433453F876
:10697400041BA34242F8041BF9D1A34B0DF13F02BF
:1069840003F1400153F8040B8B4242F8040BF9D194
:10699400FEF758BF9D4AE31C433453F8041BA3423B
:1069A40042F8041BF9D1994B0DF13F0203F1400168
:1069B40053F8040B8B4242F8040BF9D1FEF742BFA3
:1069C400934AE31C433453F8041BA34242F8041BC8
:1069D400F9D18F4B0DF13F0203F1400153F8040B41
:1069E4008B4242F8040BF9D1FEF72CBF894B0DF111
:1069F4003F0203F1400153F8040B8B4242F8040BAD
:106A0400F9D1FEF71FBF844B0DF13F0203F14001A2
:106A140053F8040B8B4242F8040BF9D1FEF712BF72
:106A24007E4B0DF13F0203F1400153F8040B8B42FE
:106A340042F8040BF9D1FEF705BF794B0DF13F0283
:106A440003F1400153F8040B8B4242F8040BF9D1D3
:106A5400FEF7F8BE734B0DF13F0203F1400153F80A
:106A6400040B8B4242F8040BF9D1FEF7EBBE6E4BDC
:106A74000DF13F0203F1400153F8040B8B4242F83D
:106A8400040BF9D1FEF7DEBE684B0DF13F0203F1B2
:106A9400400153F8040B8B4242F8040BF9D1FEF782
:106AA400D1BE634B0DF13F0203F1400153F8040BD7
:106AB4008B4242F8040BF9D1FEF7C4BE5D4B0DF1D5
:106AC4003F0203F1400153F8040B8B4242F8040BDC
:106AD400F9D1FEF7B7BE584B0DF13F0203F1400167
:106AE40053F8040B8B4242F8040BF9D1FEF7AABE0B
:106AF400524B0DF13F0203F1400153F8040B8B425A
:106B040042F8040BF9D1FEF79DBE4D4B0DF13F0247
:106B140003F1400153F8040B8B4242F8040BF9D102
:106B2400FEF790BE474B0DF13F0203F1400153F8CD
:106B3400040B8B4242F8040BF9D1FEF783BE424B9F
:106B44000DF13F0203F1400153F8040B8B4242F86C
:106B5400040BF9D1FEF776BE3C4B0DF13F0203F175
:106B6400400153F8040B8B4242F8040BF9D1FEF7B1
:106B740069BE374B0DF13F0203F1400153F8040B9A
:106B84008B4242F8040BF9D1FEF75CBE314B0DF198
:106B94003F0203F1400153F8040B8B4242F8040B0B
:106BA400F9D1FEF74FBE2C4B0DF13F0203F140012A
:106BB40053F8040B8B4242F8040BF9D1FEF742BEA2
:106BC400264B0DF13F0203F1400153F8040B8B42B5
:106BD40042F8040BF9D1FEF735BE214B0DF13F020B
:106BE40003F1400153F8040B8B4242F8040BF9D132
:106BF400FEF728BE60050020A002002060060020E9
:106C0400A00600202005002050090020900A002042
:106C1400D0080020D0070020E0020020100B002044
:106C2400A0030020E0010020100A0020A00B002097
:106C3400E00600206007002020060020D00A002083
:106C4400200700201009002060040020A005002077
:106C5400600B0020E0040020600100209008002068
:106C640050080020924B0DF13F0203F1400153F80C
:106C7400040B8B4242F8040BF9D1FEF7E3BD8D4BB4
:106C84000DF13F0203F1400153F8040B8B4242F82B
:106C9400040BF9D1FEF7D6BD874B0DF13F0203F18A
:106CA400400153F8040B8B4242F8040BF9D1FEF770
:106CB400C9BD824B0DF13F0203F1400153F8040BAF
:106CC4008B4242F8040BF9D1FEF7BCBD7C4B0DF1AD
:106CD4003F0203F1400153F8040B8B4242F8040BCA
:106CE400F9D1FEF7AFBD774B0DF13F0203F140013F
:106CF40053F8040B8B4242F8040BF9D1FEF7A2BD02
:106D0400714B0DF13F0203F1400153F8040B8B4228
:106D140042F8040BF9D1FEF795BD6C4B0DF13F021F
:106D240003F1400153F8040B8B4242F8040BF9D1F0
:106D3400FEF788BD664B0DF13F0203F1400153F8A5
:106D4400040B8B4242F8040BF9D1FEF77BBD614B77
:106D54000DF13F0203F1400153F8040B8B4242F85A
:106D6400040BF9D1FEF76EBD5B4B0DF13F0203F14D
:106D7400400153F8040B8B4242F8040BF9D1FEF79F
:106D840061BD564B0DF13F0203F1400153F8040B72
:106D94008B4242F8040BF9D1FEF754BD504B0DF170
:106DA4003F0203F1400153F8040B8B4242F8040BF9
:106DB400F9D1FEF747BD4B4B0DF13F0203F1400102
:106DC40053F8040B8B4242F8040BF9D1FEF73ABD99
:106DD400454B0DF13F0203F1400153F8040B8B4284
:106DE40042F8040BF9D1FEF72DBD404B0DF13F02E3
:106DF40003F1400153F8040B8B4242F8040BF9D120
:106E0400FEF720BD3A4B0DF13F0203F1400153F868
:106E1400040B8B4242F8040BF9D1FEF713BD354B3A
:106E24000DF13F0203F1400153F8040B8B4242F889
:106E3400040BF9D1FEF706BD2F4B0DF13F0203F110
:106E4400400153F8040B8B4242F8040BF9D1FEF7CE
:106E5400F9BC2A4B0DF13F0203F1400153F8040B36
:106E64008B4242F8040BF9D1FEF7ECBC244B0DF134
:106E74003F0203F1400153F8040B8B4242F8040B28
:106E8400F9D1FEF7DFBC1F4B0DF13F0203F14001C6
:106E940053F8040B8B4242F8040BF9D1FEF7D2BC31
:106EA4004FF4D0621849194800F0A8FFFEF7CABC95
:106EB4002002002090090020A0040020E00300200C
:106EC4001008002020010020500A0020E0050020C6
:106ED4006002002060030020A001002020030020A5
:106EE400D00900202004002060050020A00200201A
:106EF40060060020A0060020200500205009002084
:106F0400900A0020D00800204B9300082493000826
:106F14001FB50A248DE81C000A46102301460548C3
:106F2400FAF724FA04460520F9F76AFE204604B06D
:106F340010BD00BFE00B00201FB50A248DE81C0023
:106F44000A46102301460548FAF7A6FA0446052026
:106F5400F9F756FE204604B010BD00BFE00B002038
:106F640010B54023DF4A0021A020FFF7E5FF4023AE
:106F7400DD4A1946A020FFF7DFFF4023DB4A8021CA
:106F8400A020FFF7D9FF4023D94AC021A020FFF752
:106F9400D3FF4023D74A4FF48071A020FFF7CCFFE2
:106FA4004023D54A4FF4A071A020FFF7C5FF40232A
:106FB400D24A4FF4C071A020FFF7BEFF4023D04A4D
:106FC4004FF4E071A020FFF7B7FF4023CD4A4FF400
:106FD4000071A020FFF7B0FF4023CB4A4FF410719B
:106FE400A020FFF7A9FF4023C84A4FF42071A02036
:106FF400FFF7A2FF4023C64A4FF43071A020FFF7E9
:107004009BFF4023C34A4FF44071A020FFF794FF35
:107014004023C14A4FF45071A020FFF78DFF402355
:10702400BE4A4FF46071A020FFF786FF4023BC4A9C
:107034004FF47071A020FFF77FFF4023B94A4FF44B
:107044008061A020FFF778FF4023B74A4FF488619E
:10705400A020FFF771FF4023B44A4FF49061A020B1
:10706400FFF76AFF4023B24A4FF49861A020FFF76C
:1070740063FF4023AF4A4FF4A061A020FFF75CFFF9
:107084004023AD4A4FF4A861A020FFF755FF4023E9
:10709400AA4A4FF4B061A020FFF74EFF4023A84A4C
:1070A4004FF4B861A020FFF747FF4023A54A4FF4EF
:1070B400C061A020FFF740FF4023A34A4FF4C861FA
:1070C400A020FFF739FF4023A04A4FF4D061A0204D
:1070D400FFF732FF40239E4A4FF4D861A020FFF708
:1070E4002BFF40239B4A4FF4E061A020FFF724FFCD
:1070F4004023994A4FF4E861A020FFF71DFF402385
:10710400964A4FF4F061A020FFF716FF4023944AFB
:107114004FF4F861A020FFF70FFF4023914A4FF48A
:107124000061A020FFF708FF40238F4A4FF4046159
:10713400A020FFF701FF40238C4A4FF40861A020F0
:10714400FFF7FAFE40238A4A4FF40C61A020FFF7B0
:10715400F3FE4023874A4FF41061A020FFF7ECFEB2
:107164004023854A4FF41461A020FFF7E5FE402335
:10717400824A4FF41861A020FFF7DEFE4023804AC4
:107184004FF41C61A0207F4CFFF7D6FE40237E4ABB
:107194004FF42061A020FFF7CFFE40237B4A4FF439
:1071A4002461A020FFF7C8FE224601234FF4286182
:1071B400A020FFF7C1FE621C042340F68421A02016
:1071C400FFF7BAFE621D042340F68821A020FFF7D2
:1071D400B3FE04F10902032340F68C21A020FFF73B
:1071E400ABFE04F10C0203234FF42961A020FFF746
:1071F400A3FE04F10F02032340F69421A020FFF71D
:107204009BFE04F11202032340F69821A020FFF70D
:1072140093FE04F11502012340F69C21A020FFF700
:107224008BFE04F1160204234FF42A61A020FFF719
:1072340083FE04F11A02042340F6A421A020FFF7E0
:107244007BFE04F11E02032340F6A821A020FFF7D1
:1072540073FE04F12102032340F6AC21A020FFF7C2
:107264006BFE04F1240203234FF42B61A020FFF7EB
:1072740063FE04F12702464C032340F6B421A02008
:10728400FFF75AFE2246012340F6B821A020FFF75B
:1072940053FE621C042340F6B921A020FFF74CFEE4
:1072A400621D032340F6BD21A020FFF745FE04F133
:1072B400080201234FF42C61A020FFF73DFE04F1E6
:1072C4000902042340F6C121A020FFF735FE04F192
:1072D4000D020323BDE8104040F6C521A020FFF7AE
:1072E4002BBE00BFD0070020E0020020100B0020BE
:1072F400A0030020E0010020100A0020A00B0020C1
:10730400E00600206007002020060020D00A0020AC
:10731400200700201009002060040020A0050020A0
:10732400600B0020E0040020600100209008002091
:10733400500800202002002090090020A004002012
:10734400E00300201008002020010020500A002043
:10735400E00500206002002060030020A00100205E
:1073640020030020D0090020200400206005002014
:10737400A002002060060020A006002020050020B6
:1073840050090020A6070020900A0020D008002001
:10739400500B002010B514460A230248FAF7CEFE1B
:1073A400204610BD380C002008B502680B4B9A42E9
:1073B40012D10B4A1368013313600A4A136801336C
:1073C4001360094B1B783BB1FBF72EFC132881BFDC
:1073D400064A13680133136008BD00BF0010004063
:1073E400C8000020C4000020CC000020C000002001
:1073F40002680E4B9A4217D10D490E4A0978137848
:107404000D48EB29C15404BF01200C4903F10103C9
:10741400DBB208BF08703F2B88BF002304491370F8
:1074240007480122FAF7E6BE704700BF0048004053
:10743400780C00207B0C0020BC0C0020340C0020B5
:10744400380C0020014B1870704700BF340C00202A
:1074540010B592B03022002106A800F0C6FC142218
:10746400002101A800F0C1FC0123099310230A9311
:107474000D230E93C32302240F93042306A8119310
:1074840006940C941094FAF719F90F23019300232E
:1074940003934FF4A05304934FF48053032101A8A2
:1074A40002940593FAF7A6FA12B010BD2DE9F04F35
:1074B4000024A7B008AD642200210DA800F095FCBB
:1074C400F9F776FBFFF7C4FF14220021284600F0E9
:1074D4008CFCB44B00941A6B47F63D7142F01002D9
:1074E4001A631A6BB04802F010020092009A0194D9
:1074F4001A6B012742F004021A631A6B4FF4E13A43
:1075040002F004020192019A02941A6B4FF00C09E2
:1075140042F020021A631A6BDFF8E08202F02002C4
:107524000292029A03941A6BA04E42F080021A63EC
:107534001A6B02F080020392039A04941A6B42F0CD
:1075440001021A631A6B02F001020492049A059470
:107554001A6B42F002021A631A6B02F002020592DD
:10756400059A06941A6B42F040021A631A6B02F0F1
:1075740040020692069A07941A6B42F008021A63B4
:107584001B6B224603F008030793079BF9F7AEFC35
:1075940022464DF630418648F9F7A8FC22464EF6BD
:1075A40007018448F9F7A2FC22464FF40F61824890
:1075B400F9F79CFC224640F2E1218048F9F796FC59
:1075C400224647F6FC217E48F9F790FC2246CF215B
:1075D4007C48F9F78BFC47F63D73294672480893BB
:1075E4000A940B940997F9F795FB4DF63043294615
:1075F4006F4808930A940B940997F9F78BFB4EF69E
:10760400070329466B4808930A940B940997F9F7E2
:1076140081FB4FF4E07329466648089309940A9461
:10762400F9F778FB0E2329466148089309940A94D4
:10763400F9F770FB4FF40F6329465F4808930A94E7
:107644000B940997F9F766FB40F2E12329465B485E
:1076540008930A940B940997F9F75CFB47F6FC230B
:107664002946574808930A940B940997F9F752FB53
:10767400CF232946534808930A940B940997F9F7A2
:1076840049FB5148514B846080E80804C46004619C
:107694008461C461C0F81490FAF722FD41F26F735B
:1076A4004B4A404688E80C0009230894C8F80C307B
:1076B4006C60C8F80840C8F81840FAF783FB2946FC
:1076C400404608940994FAF797FB42484249434BD1
:1076D400846080E80A004FF48043C460036144611D
:1076E4008461C4610462F9F7D3FD3D4B304686E8FA
:1076F4000804B460F4603461B461F461C6F81490B1
:10770400FAF7EEFC224621462520F9F79BFA2520BC
:10771400F9F7CCFA224621463620F9F793FA3620B7
:10772400F9F7C4FA224621462720F9F78BFA2720D5
:10773400F9F7BCFA4046FAF72BFA3A46294930469B
:10774400FAF758FD284800F0ABFA284B21461B688D
:10775400986800F0CFFBFFF703FCFAF7DBFF204645
:10776400FBF74EFD224B0DAC03F140062246186890
:107774005968083303C2B3421446F7D1FDF7E6F85B
:107784001C4EDFF82C80184B9B68002B67DC337889
:10779400012B68D1184B1B68642B64D9DFF8609007
:1077A40030E000BF0038024000100240380C0020D6
:1077B400000802400014024000000240000402409D
:1077C40000180240000C02407C0C00200010014014
:1077D40000100040E00B0020005C0040801A06000E
:1077E40000480040780C0020400D002004000020D8
:1077F40020060020340C0020C8000020FC0C0020CF
:10780400CD000020454F99F8021009F1010009EB61
:1078140001030231DA78C9B200F0B1F84C4600280D
:1078240071D1DFF820B13B7800F1010AC0B298426F
:1078340063D33B4800F056FB99F8022039481444BE
:10784400E178053200F0DAFA40220021364800F0EF
:10785400CCFA002038703070FAF7D4FD93E733483F
:1078640000F024FA8FE7FAF7D3FD012896D0304CC4
:107874002368C82B08D92F4800F0C0FA2E4B18787B
:10788400FBF7BEFC002323602C4C2368B3F5FA7F7E
:107894007FF679AF2846FCF723FD95E80300FCF753
:1078A40053FDBE238DF834306D238DF83530082315
:1078B40028688DF83630AB88CDF837000A210DF1F1
:1078C4003500ADF83B3000F03FF89DF8363026AA7D
:1078D4001344EB228DF83F0003F8602C9DF836101A
:1078E4000DA80531C9B2FCF77DFD4FF400414046B7
:1078F400F9F701FB0023236045E7215C584600F0BB
:107904007DFA50468FE7012803D14846FDF70AFF68
:107914009AE70B4800F0E6FA96E700BF0E01002054
:107924009F93000866930008CD000020380C0020C7
:10793400C0000020A19300080D010020C400002015
:10794400939300086093000810B5FF230446221A9D
:10795400D2B2914201D8184610BD14F8012B5340FD
:10796400082213F0800F02F1FF324FEA430318BFDD
:1079740083F0310312F0FF02DBB2F2D1E7E730B556
:10798400FF2305462C1AE4B2A14203D89B1A58429D
:10799400584130BD15F8014B6340082413F0800FA3
:1079A40004F1FF344FEA430318BF83F0310314F0AA
:1079B400FF04DBB2F2D1E5E7002182B00B4B00916A
:1079C4005A6C42F480425A645A6C02F48042009227
:1079D400009A01911A6C42F080521A641B6C03F0F5
:1079E40080530193019B02B0704700BF00380240EE
:1079F4002DE9F043044689B01422002103A800F0C5
:107A0400F4F92268224B9A423FD10025214C00957B
:107A1400236B4FF0120943F004032363236B4FF0ED
:107A2400010803F004030093009B0195236B0327D3
:107A340043F001032363236B042603F00103019342
:107A4400019B4FF4007303A913480393CDF81090DE
:107A5400CDF8148006970796F9F75CF94FF4807314
:107A640003A90E480393CDF81090CDF8148006971F
:107A74000796F9F74FF90295236C43F40003236446
:107A8400236C03F400030293029B09B0BDE8F08366
:107A9400005C004000380240000802400000024040
:107AA4000268094B82B09A420BD100230193074B21
:107AB4001A6C42F010021A641B6C03F01003019359
:107AC400019B02B0704700BF001000400038024024
:107AD400142210B504468AB00DEB0200002100F018
:107AE40084F92368284A934226D10021274B019127
:107AF4005A6C274842F010025A645A6C02F0100281
:107B04000192019A02911A6B05A942F001021A63CB
:107B14001B6B03F001030293029B4FF4C0630593B4
:107B2400022306930123079303230893072309934E
:107B3400F9F7F0F80AB010BD164A9342FAD10021C1
:107B4400124B03911A6C144842F480221A641A6C82
:107B540002F480220392039A04911A6B05A942F05D
:107B640002021A631B6B03F002030493049B4FF499
:107B74004063059302230693012307930323089389
:107B840007230993D4E700BF0010014000380240E6
:107B94000000024000480040000402407047FEE735
:107BA400FEE7FEE7FEE7704770477047F9F71AB83B
:107BB4000148FAF77FBB00BF7C0C002013B50A4CC8
:107BC40023681A68920604D559682046C9B200F0A1
:107BD40093F80023019323681A6801925B68019368
:107BE400019B02B010BD00BF380C00200148F9F71A
:107BF400DEBF00BFFC0C002070B50E4615460C46D7
:107C0400A31B9D4201DC284670BDAFF3008004F83D
:107C1400010BF5E708B50A4B0246196809B9094989
:107C240019606946186802448A4206D900F0A8F827
:107C34000C2303604FF0FF3008BD1A6008BD00BF7D
:107C4400100100205C1500204FF0FF3070474FF406
:107C5400005300204B60704701207047002070479C
:107C640000210C4B1A6842F001021A6099601A68EC
:107C740022F0847222F480321A60074A5A601A6829
:107C840022F480221A604FF00062D960034B9A609C
:107C9400704700BF003802401030002400ED00E0BF
:107CA40000234360036083607047000010B50F4AEF
:107CB4001178C9B24B1CDBB213700D4B5A6803F137
:107CC4000C00145C0132B2F5806FA8BF00225A6028
:107CD4009A680848013A44549A6012B90120FFF79F
:107CE400B1FBBDE810400120F8F78ABF0E01002067
:107CF400400D0020CD00002038B50B4C0D46A36884
:107D0400B3F5806F01DBFFF7D1FF23685A1CB2F58E
:107D1400806F23441D7308BF0023226008BF2360C3
:107D2400A3680133A36038BD400D0020DFF834D0D0
:107D3400002103E00C4B5B58435004310B480C4BBF
:107D440042189A42F6D30B4A02E0002342F8043B5D
:107D5400094B9A42F9D3FFF783FF00F017F8FFF7B6
:107D6400A5FB704700000220749400080000002066
:107D740068000020680000205C150020FEE7000079
:107D8400014B1868704700BF0400002070B500253F
:107D94000C4E0D4CA41BA410A54209D101F01AFAF3
:107DA40000250A4E0A4CA41BA410A54205D170BD9F
:107DB40056F8253098470135EEE756F825309847B0
:107DC4000135F2E76C9400086C9400086C94000888
:107DD4007094000810B5431E0A44914200D110BDAE
:107DE40011F8014B03F8014FF7E7034602449342AD
:107DF40000D1704703F8011BF9E700000FB40A4BE8
:107E040013B51C6824B1A36913B9204600F006FB1E
:107E140005AB049AA1682046019300F017FE02B056
:107E2400BDE8104004B070470400002070B50E4651
:107E3400054618B183690BB900F0F0FAAB69AC6878
:107E440013B9284600F0EAFA234B9C4217D16C6818
:107E5400A3891B071DD52369DBB1013EA36816F86E
:107E6400011F013BA360E9B9002B2EDA22460A2147
:107E7400284600F021F9013011D00A2070BD174BBB
:107E84009C4201D1AC68E3E7154B9C4208BFEC6807
:107E9400DEE72146284600F061F90028DDD04FF0E6
:107EA400FF3070BD002B04DAA269934206DB0A2975
:107EB40004D023685A1C22601970CFE72246284652
:107EC40000F0FAF80130C9D1E9E70A2023685A1C06
:107ED4002260187070BD00BFF09300081094000871
:107EE400D0930008024B01461868FFF79FBF00BFFC
:107EF4000400002000294FF480630CBF02220022FA
:107F040000F000B82DE9F7431D46514B04461E68A6
:107F14000F46904626B1B36913B9304600F07EFA95
:107F24004C4B9C4252D17468B8F1020F06D0B8F1A0
:107F3400010F00F28980002DC0F286802146304670
:107F440000F002FA616B41B104F14403994202D09A
:107F5400304600F059FB002363630023A361636090
:107F6400A3891B0603D52169304600F04DFBA38984
:107F7400B8F1020F23F44A6323F00303A3815DD015
:107F840001AB6A462146304600F0D2FAA389184371
:107F9400A0812DBB009D284600F02EFB074600283B
:107FA4004ED1DDF80090A9453CD14FF0FF30A389B4
:107FB40043F00203A3810023A36004F14703236079
:107FC40023610123636103B0BDE8F083224B9C422B
:107FD40001D1B468A8E7214B9C4208BFF468A3E729
:107FE400002FD8D0B36913B9304600F017FAB8F1AE
:107FF400010F08BFA389276004BF43F00103A381D5
:10800400A389276113F0080065611BD013F00100F8
:108014004FF000031FBF6D42A360A561184608BF5F
:10802400A560D0E7484600F0E7FA07460028BCD030
:10803400A3894D4643F08003A381D3E70020B6E72C
:10804400A946F5E7A060BEE74FF0FF30BBE700BFED
:1080540004000020F093000810940008D093000856
:108064000EB44FF4027100B59CB0ADF814106FF06B
:108074000041049107914FF6FF711DAB02900690E9
:10808400084853F8042BADF81610006802A90193B0
:1080940000F0C0FB0022029B1A701CB05DF804EBD8
:1080A40003B0704704000020034611F8012B03F8C5
:1080B400012B002AF9D17047F8B50E46144605463F
:1080C40018B183690BB900F0A9F9214B9C422AD15C
:1080D4006C68A369A360A3891A072ED5236963B3C7
:1080E40023692068F6B2C01A63693746984204DBF4
:1080F4002146284600F028F928BBA3680130013B3B
:10810400A36023685A1C22601E706369984204D0DD
:10811400A389DB0719D50A2E17D12146284600F07A
:1081240013F990B10FE00B4B9C4201D1AC68D0E73E
:10813400094B9C4208BFEC68CBE72146284600F077
:108144000DF80028CCD04FF0FF373846F8BD00BFFB
:10815400F093000810940008D0930008324B70B5D7
:108164001D6806460C4625B1AB6913B9284600F0D4
:1081740055F92E4B9C420FD16C68B4F90C309AB26D
:1081840015072CD4D00611D40922326043F04003E1
:10819400A3814FF0FF3070BD254B9C4201D1AC68E8
:1081A400EBE7244B9C4208BFEC68E6E7510712D585
:1081B400616B41B104F14403994202D0304600F0AE
:1081C40023FA00236363A38923F02403A3810023F8
:1081D400636023692360A38943F00803A3812369AF
:1081E4004BB9A38903F42073B3F5007F03D0214670
:1081F400304600F0C1F9A28912F001030CD000232B
:10820400A36063695B42A361236953B9B4F90C3079
:1082140013F08000BAD170BD920758BF6369A360A0
:10822400F2E70020F7E700BF04000020F093000805
:1082340010940008D09300088A892DE9F04105467E
:1082440010070C465AD44B68002B05DC0B6C002B32
:1082540002DC0020BDE8F081E66A002EF9D000239C
:1082640012F480522F682B6033D0606DA3895A07B3
:1082740005D56368C01A636B0BB1236CC01A002365
:108284000246E66A216A2846B047431CA38906D100
:1082940029681D294BD82B4ACA40D60747D5002246
:1082A40062602269D904226004D5421C01D12B6882
:1082B40003B96065616B2F600029CAD004F14403DF
:1082C400994202D0284600F09FF900206063BDE87F
:1082D400F081216A01232846B047411CC6D12B688E
:1082E400002BC3D01D2B01D0162B01D12F60B0E77A
:1082F400A38943F04003A381BDE8F0810F69002FF7
:10830400A7D0930718BF00230E6808BF4B69A6EBDC
:1083140007080F608B60B8F1000F9ADD43463A46B8
:10832400216A2846A66AB047002807DCA38943F0DF
:108334004003A3814FF0FF30BDE8F0810744A8EB70
:108344000008E8E70100402038B50B6905460C46F3
:10835400DBB118B183690BB900F060F80C4B9C4297
:1083640009D16C68B4F90C307BB121462846BDE8CC
:108374003840FFF761BF074B9C4201D1AC68F1E77D
:10838400054B9C4208BFEC68ECE7002038BD00BFF9
:10839400F093000810940008D0930008014900F0FD
:1083A400A9B800BF4D830008002310B5044603603C
:1083B4004360836081814366C28103614361836159
:1083C400194608225C30FFF710FD054B24626362F6
:1083D400044BA362044BE362044B236310BD00BF50
:1083E400CD8F0008EF8F0008279000084B900008FD
:1083F40070B568254A1E55430E4605F1740100F018
:108404004FF9044640B1002180E842000C30A060DE
:1084140005F16802FFF7E9FC204670BD836910B5D9
:10842400044633BB8364C3640365124B124A1B685E
:108434008262984204BF0123836100F01FF86060E8
:10844400204600F01BF8A060204600F017F8002238
:10845400E06004216068FFF7A7FF01220921A068FA
:10846400FFF7A2FF02221221E068FFF79DFF01231C
:10847400A36110BDCC930008A1830008F8B51C4B80
:1084840007461E68B36913B93046FFF7C7FF48367D
:10849400B4687368013B03D5336833B13668F7E7D2
:1084A400B4F90C506DB16834F4E704213846FFF791
:1084B4009FFF30600028F1D10C2304463B60204626
:1084C400F8BD4FF6FF73E38101236566A381256040
:1084D400A560656025616561A5610822294604F1EE
:1084E4005C00FFF782FC6563A563A564E564E6E7C9
:1084F400CC9300082DE9F84380468946002600F114
:10850400480414B93046BDE8F883A5686768013F9C
:1085140001D52468F5E7AB89012B07D9B5F90E30ED
:10852400013303D029464046C84706436835EEE781
:1085340070B50E46B1F90E1090B0002914461D46D0
:1085440007DA00232B60B3891A0610D44FF4806332
:108554000EE001AA00F09EFD0028F2DB029A02F46C
:108564007042A2F500535A425A412A60EEE7402372
:108574000020236010B070BD8B8973B59D0706463B
:108584000C4607D504F1470323602361012363618B
:1085940002B070BD01AB6A46FFF7CAFF00990546F9
:1085A400304600F07DF848B9B4F90C309A05EFD4A0
:1085B40023F0030343F00203A381E3E70D4BB3620B
:1085C400A389206043F08003A381009B2061636141
:1085D400019B5BB1B4F90E10304600F06DFD28B17B
:1085E400A38923F0030343F00103A381A3891D435B
:1085F400A581CDE7A1830008024B0146186800F06D
:108604004FB800BF0400002038B50546002943D008
:1086140051F8043C0C1F002BB8BFE41800F096FD81
:108624001E4A1368104633B9636014602846BDE8D7
:10863400384000F08CBDA3420BD9216862189342E4
:1086440001BF1A685B685218226063600460EDE73A
:1086540013465A680AB1A242FAD919685818A042B6
:108664000BD120680144581882421960DED1106889
:108674005268014419605A60D8E702D90C232B6070
:10868400D4E7206821188A4201BF1168526809188A
:10869400216062605C60C9E738BD00BF140100203E
:1086A40070B5CD1C25F0030508350C2D38BF0C25FD
:1086B400002D064601DBA94203D90C2333600020B8
:1086C40070BD00F043FD234A1468214691B9224C41
:1086D40023681BB9304600F067FC20602946304609
:1086E40000F062FC431C26D10C233046336000F0BA
:1086F4002EFDE4E70B685B1B1AD40B2B0FD90B6020
:10870400CC18CD50304600F022FD04F10B00231D9F
:1087140020F00700C31A1BD05A42E25070BD8C42AD
:108724000BBF63684B681360636018BF0C46E9E7CE
:108734000C464968CAE7C41C24F00304A04205D0CF
:10874400211A304600F030FC0130CDD02560D9E745
:1087540070BD00BF14010020180100202DE9F0476E
:108764008E6882469E420C469146984635D88A8940
:1087740012F4906F31D00223256809696F1A656974
:1087840005EB450595FBF3F508F101033B449D42D8
:1087940038BF1D46530531D52946FFF781FF0646EC
:1087A40050B90C23CAF80030A3894FF0FF3043F0CE
:1087B4004003A381BDE8F0873A462169FFF70AFB2D
:1087C400A38923F4906343F08003A38126613E448C
:1087D400266046466561ED1BA560464528BF4646B2
:1087E40049463246206800F097FCA36800209B1B92
:1087F400A36023681E442660BDE8F0872A4600F083
:10880400A7FC06460028E1D121695046FFF7FCFE8B
:10881400C7E700002DE9F04F9DB003938B89804694
:108824001C060D4616460FD50B696BB94021FFF7A0
:1088340037FF2860286128B90C23C8F800304FF0AE
:10884400FF30C4E040236B610023099320238DF89B
:10885400293030234FF0010B8DF82A3037463C463F
:1088640014F8013B002B3CD1B7EB060A0BD053465E
:10887400324629464046FFF771FF013000F0A280DE
:10888400099B534409933B78002B00F09B80002301
:108894004FF0FF3204930793059206938DF85330FB
:1088A4001A9305222178504800F028FC671C049B89
:1088B400D8B9D90644BF20228DF853201A0744BFE3
:1088C4002B228DF8532022782A2A16D000210A2040
:1088D400079A27463B780134303B092B50D9C9B15C
:1088E40011E0252BC0D02746B9E73F4A3C46801A01
:1088F4000BFA00F018430490D3E7039A111D126891
:108904000391002A01DB079204E0524243F0020380
:10891400079204933B782E2B0DD17B78791C2A2B5C
:1089240032D1039B02371A1D1B680392002BB8BF78
:108934004FF0FF3305932D4C03223978204600F085
:10894400DDFB38B14023001B03FA00F0049B013720
:10895400034304933978062225487E1C8DF8281099
:1089640000F0CCFB002835D0224BFBB9039B073326
:1089740023F0070308330393099B4B4409936DE7E2
:1089840000FB02320121A4E700230A2418460593C0
:108994000F463A780131303A092A03D9002BCAD05C
:1089A4000590C8E704FB00200123F1E703AB009323
:1089B4002A46114B04A94046AFF30080B0F1FF3FB3
:1089C4008146D9D1AB895B063FF539AF09981DB013
:1089D400BDE8F08F03AB00932A46074B04A9404639
:1089E40000F0C2F9EAE700BF3094000836940008AA
:1089F4003A9400080000000061870008936810B4EE
:108A0400013B002B936008DA9469A34202DBCBB2EA
:108A14000A2B02D110BCFFF74FBB1368581C10601F
:108A24001970C8B210BC7047F8B506460F46144614
:108A3400D518AC4201D1002007E03A4614F8011BD6
:108A44003046FFF7DBFF431CF3D1F8BD2DE9F04FAF
:108A54009DB00C4617460393064618B183690BB9BB
:108A6400FFF7DCFC7C4B9C4257D17468A389180740
:108A74005DD52369002B5AD00023099320238DF858
:108A8400293030234FF0010B8DF82A30B846454683
:108A940015F8013B002B55D1B8EB070A0BD0534610
:108AA4003A4621463046FFF7BFFF013000F0C4804C
:108AB400099B5344099398F80030002B00F0BC80C4
:108AC40000234FF0FF3204930793059206938DF829
:108AD40053301A9305222978604800F00FFB05F102
:108AE4000108049B002831D1D90644BF20228DF807
:108AF40053201A0744BF2B228DF853202A782A2AA0
:108B04002CD000210A20079AA84698F80030013595
:108B1400303B092B6DD971B326E0514B9C4201D1F6
:108B2400B468A3E74F4B9C4208BFF4689EE7214614
:108B34003046FFF713FB00289ED04FF0FF301DB0E6
:108B4400BDE8F08F252BA7D0A846A0E7434A4546A9
:108B5400801A0BFA00F018430490BBE7039A111D26
:108B640012680391002A01DB079204E0524243F0A9
:108B740002030792049398F800302E2B10D198F832
:108B8400013008F101012A2B37D1039B08F10208B7
:108B94001A1D1B680392002BB8BF4FF0FF330593D7
:108BA400314D032298F80010284600F0A7FA40B18E
:108BB4004023401B03FA00F0049B08F1010803431F
:108BC400049398F800100622284808F101078DF84C
:108BD400281000F093FA002834D0254B03BB039BE4
:108BE400073323F0070308330393099B4B4409938A
:108BF4004CE700FB0232012186E700230A251846D0
:108C04000593884698F800200131303A092A03D99F
:108C1400002BC5D00590C3E705FB00200123F0E736
:108C240003AB00932246134B04A93046AFF30080F4
:108C3400B0F1FF3F8146D8D1A3895B063FF57DAFF4
:108C440009987CE703AB009322460A4B04A93046FB
:108C540000F08AF8ECE700BFF093000830940008B5
:108C640010940008D0930008369400083A94000841
:108C7400000000002D8A00082DE9F04791461F46A8
:108C84008A680B6906469342B8BF1346C9F8003098
:108C940091F843200C46DDF8208012B10133C9F865
:108CA40000302368990642BFD9F800300233C9F86E
:108CB4000030256815F0060507D104F1190AE368A8
:108CC400D9F800209B1A9D422ADB94F8433022688D
:108CD400003318BF012392062FD404F1430239460E
:108CE4003046C047013022D02368E56803F006030C
:108CF400042B18BF0025D9F800204FF0000908BF45
:108D0400AD1AA368226908BF25EAE5759342C4BF7A
:108D14009B1AED181A344D451BD10020BDE8F0878D
:108D24000123524639463046C047013003D14FF043
:108D3400FF30BDE8F0870135C1E73020E11881F844
:108D440043005A1C94F845102244023382F843101D
:108D5400C3E70123224639463046C0470130E6D0F6
:108D640009F10109D7E700002DE9F04317460A7E0F
:108D740085B06E2A984606460C460C9B01F1430EBC
:108D840000F0BC801AD8632A2ED00AD8002A00F03A
:108D9400C880582A00F08A8004F1420584F84220F1
:108DA4002AE0642A01D0692AF6D121681A6811F0F0
:108DB400800F23D0111D1960136827E0732A00F077
:108DC400B48008D86F2A2AD0702AE5D10A6842F004
:108DD40020020A6003E0752A21D0782ADCD17822A7
:108DE4006F4984F8452064E01A6801F14205111DB9
:108DF4001960136884F842300123A3E011F0400F96
:108E040002F104011960D7D0B2F90030002B03DA63
:108E14002D225B4284F8432062490A2217E020682D
:108E2400196810F0800F03D0081D18600B6806E065
:108E340010F0400F01F104001860F7D00B886F2A7E
:108E440014BF0A2208225749002084F843006568A9
:108E5400002DA560C0F29C80206820F004002060F2
:108E6400002B3FD1002D40F095807546082A0BD188
:108E74002368DA0708D5236962689A42DEBF302383
:108E840005F8013C05F1FF35AEEB05032361CDF890
:108E940000803B4603AA21463046FFF7EDFE013031
:108EA40055D14FF0FF3005B0BDE8F08381F845207F
:108EB4003C492268186812F0800F00F104051D6017
:108EC40001D0036802E05506FBD50388D00744BFF0
:108ED40042F0200222601BB9226822F020022260A4
:108EE4001022B1E77546B3FBF2F002FB1033CB5C02
:108EF40005F8013D03460028F5D1B7E708681A686C
:108F040010F0800F496904D0101D186013681960AF
:108F140007E010F0400F02F1040018601368F6D067
:108F24001980002375462361B1E71A68111D196081
:108F3400156800216268284600F0E0F808B1401B7B
:108F4400606063682361002384F843309FE72369EA
:108F54002A4639463046C0470130A2D023689B07D1
:108F640007D5002504F11909E368039A9B1A9D4269
:108F740005DBE068039B9842B8BF184693E70123DA
:108F84004A4639463046C04701308AD00135EBE7BE
:108F9400002BA7D10B7804F1420584F8423065E731
:108FA400529400084194000838B50023054C054646
:108FB40008462360FEF72EFE431C02D1236803B14A
:108FC4002B6038BD5815002010B50C46B1F90E10B1
:108FD40000F0E4F80028ABBF636DA3891B1823F4E9
:108FE4008053ACBF6365A38110BD2DE9F0411F46DA
:108FF4008B890546DB050C46164605D5022300225F
:10900400B1F90E1000F068F8A389324623F48053B6
:10901400A381B4F90E103B462846BDE8F04100F0A8
:1090240017B810B50C46B1F90E1000F055F8431CF2
:10903400A38915BF606523F4805343F48053A3814F
:1090440018BFA38110BDB1F90E1000F013B80000D1
:1090540038B50546084611460022054C22601A46DA
:10906400FEF798F9431C02D1236803B12B6038BD85
:109074005815002038B50023054C054608462360E2
:10908400FEF7E2FD431C02D1236803B12B6038BD17
:109094005815002038B50023064C054608461146ED
:1090A4002360FEF7D4FD431C02D1236803B12B6077
:1090B40038BD00BF5815002038B50023054C0546BF
:1090C40008462360FEF7C8FD431C02D1236803B1A0
:1090D4002B6038BD5815002038B5054608461146A2
:1090E4000022054C22601A46FEF7B8FD431C02D14B
:1090F400236803B12B6038BD5815002010B5C9B2E0
:1091040002449042034601D1002010BD1C78013076
:109114008C42F6D1184610BD884210B501EB02030B
:1091240003D8421E99420CD110BD9842F9D281183D
:10913400D21AD34200D110BD13F8014D01F8014DEC
:10914400F7E711F8014B02F8014FEBE7704770475E
:10915400F8B5074614460E4621B91146BDE8F84055
:10916400FFF79EBA22B9FFF74FFA25462846F8BD05
:1091740000F026F884420FD921463846FFF790FACA
:1091840005460028F2D031462246FEF723FE31463A
:109194003846FFF739FAE9E73546E7E738B50546D3
:1091A400084611460022054C22601A46FEF724FDAB
:1091B400431C02D1236803B12B6038BD581500202D
:1091C40051F8040C0028A0F10400BCBF0B58C018CF
:1091D40070470000F8B500BFF8BC08BC9E46704755
:0C91E400F8B500BFF8BC08BC9E46704700
:1091F0004368616E6E656C2053657474696E6700B8
:10920000707265737320616E7920427574746F6E2D
:109210000064617461203A2025662020206F666614
:10922000736574203A202025660D0A00202032380C
:109230007E32382E352047487A20200020203238D0
:109240002E357E32392047487A2000202032397E60
:1092500032392E352047487A2000202032392E35E9
:109260007E33302047487A200020202020322E34C0
:1092700047487A20202020200020202020352E382A
:1092800047487A20202020200020204120436820C9
:109290003135304D487A2000202020202530362ED0
:1092A0003266202020644200202020412043682094
:1092B0003330470020202041204368616E6E656C8A
:1092C000202020002020202053657474696E6700E0
:1092D0002020204120436820574946492020002073
:1092E0002042204368203135304D487A200020202C
:1092F000204220436820333047002020422043682A
:10930000616E6E656C0020204220436820574946FC
:1093100049202000437269746963616C2045727250
:109320006F720D005B4572726F72205D44656661FD
:109330006C757420696E2025732020202020204C1D
:10934000494E45203A2564200D0A00417474656E2B
:109350005F4F7065726174655F4D656D5F52570058
:10936000253032782000434845434B53554D5F45E7
:1093700052524F52202052656376435243203A2086
:109380002530327820202C20696E64657820256491
:109390000D0A00576861742048617070656E3F0D5A
:1093A000004C4F4E47204B45592050524553530DCA
:1093B0006D00000000000000000001020304060729
:1093C000080900000000010203040000080000205A
:1093D000000000000000000000000000000000008D
:1093E000000000000000000000000000000000007D
:1093F000000000000000000000000000000000006D
:10940000000000000000000000000000000000005C
:10941000000000000000000000000000000000004C
:10942000000000000000000000000000000000003C
:10943000232D302B2000686C4C006566674546473D
:1094400000303132333435363738394142434445C0
:10945000460030313233343536373839616263642F
:04946000656600003D
:089464004874FF7F01000000C5
:04946C00A90100084A
:04947000850100086A
:109474000024F4000800002000000000F09300081D
:1094840010940008D09300080000000000000000C1
:1094940000000000000000000000000000000000C8
:1094A40000000000000000000000000000000000B8
:1094B40000000000000000000000000000000000A8
:1094C4000000000000000000000000000000000098
:0894D400000000000000000090
:0400000508007D3141
:00000001FF
